:020000040800F2
:10500000A0300020D550000855A5000829980008B8
:105010000000000000000000000000000000000090
:10502000000000000000000000000000B1AC00081B
:10503000000000000000000057A50008DDB20008D5
:10504000E7500008E7500008E7500008E750000864
:10505000E75000081F630008E75000082F630008AE
:1050600000000000E7500008E7500008E750000883
:10507000E7500008AD9B0008E7500008E750000823
:10508000E7500008E7500008E75000080000000063
:10509000E7500008E7500008E7500008E750000814
:1050A000E7500008E7500008E750000891C00008EA
:1050B000A1C00008ED9C00080000000000000000F6
:1050C0000348854600F0D6FC0048004715D000088C
:1050D000A03000200448804704480047FEE7FEE770
:1050E000FEE7FEE7FEE7FEE79DB30008C1500008BB
:1050F00030B50B46014600202022012409E00D4670
:10510000D5409D4205D31D469540491B25469540F7
:1051100040191546521E002DF1DC30BDF0B51FB40C
:105120000646002082B005464024019100901BE015
:10513000019922460F46304600F080FB049A059BF9
:10514000801A994110D310461946224600F066FB9A
:10515000361A8F410197224601200021009F00F05E
:105160005DFB38184D4100902046641E0028DFDCAE
:10517000019B00982946324607B0F0BD03460B4319
:105180009B0703D009E008C9121F08C0042AFAD2FD
:1051900003E00B780370401C491C521EF9D2704783
:1051A000D2B201E00270401C491EFBD270470022BF
:1051B000F6E710B513460A4604461946FFF7F0FF16
:1051C000204610BD30B505462A460B4610781C789F
:1051D000521C5B1C002801D0A042F7D0002C03D049
:1051E000002802D06D1CEFE7284630BD421C017834
:1051F000401C0029FBD1801A704730B504460020BE
:10520000034600E05B1C934203D2E05CCD5C401B94
:10521000F8D030BD70B5064607F03AFA0468054686
:105220000A220021304600F02DFB2C6070BDF8B53D
:1052300002464A40D40F42004B0052085B089A4293
:1052400002D20246084611464A0023D0C30D4A0046
:10525000DDB2120EAD1A202D35DA49020126490AB7
:10526000F6058A19002C00D0524220214F1B11460E
:10527000B9402A411018C20D9A4221D0002C17D0F3
:10528000012D08DCDA05801AD20F8019D207DBB2B3
:1052900000F038FBF8BDDA05801A012340001B0638
:1052A000C01880185A428018CA0F1043490007E0FE
:1052B0004908C2071143DA05801A8019400880188E
:1052C00000F018FBF8BD61000122511A001BF7E73E
:1052D0000122D2075140AAE70122D2075040A6E797
:1052E000024670B54A40D30FDB0740002DD04A007C
:1052F0002AD0010E140E000212020919400A520AA5
:105300008418E50104465443000A120A2E0450434F
:10531000A4194219200CC543AA18120C0125AD038B
:10532000521C521912047F39240400D0521C10431D
:1053300001D44000491EC2B20C06C0092018401C0E
:105340004008802A02D003E0002070BD40084000E1
:10535000002900DA0020184370BD70B502464A40AB
:10536000D50F40004A00ED0740085208002814D02D
:10537000002A12D0C40DD30D41020120C0055202F3
:10538000490A520AE41A091812187D34914201D3CD
:10539000641C00E04900002C01DA002070BD0023ED
:1053A000914201D3891A0343400849000028F7D1EC
:1053B00000290AD0914202D10121C90705E091429A
:1053C00001D2012101E00121C943E005C0184019C3
:1053D00000F090FA70BD420005D04200120E524219
:1053E0008A4201DB00207047C90508187047000099
:1053F000F0B507460846584087B0C00F04904800F3
:105400000E46590040084908BC1A884105D2384662
:1054100031461E4617460B460246580040081043C8
:105420004CD0300D039040055900400D490D0590BA
:10543000401A0290402872DA18030121000B090576
:105440000843019004980092002805D00199524227
:105450000020884100920190029840210A1A019987
:10546000009800F0DBF905460C466B4607CB00F0D0
:10547000F6F9C0197141039A0E0D0023D717564053
:105480001A467A40164344D0049A002A2DD0029A34
:10549000012A039A15DC1205C01A9141012636052E
:1054A000001C7141D20F059ED20700930192029613
:1054B0002A46234600F06CFA07B0F0BD3846314664
:1054C000FAE71605224A0F46B218C01AB741012161
:1054D0000905001C4F4100187F41114618187941F9
:1054E000E20F10436D19644113E0E2076D081543A4
:1054F0006408C2071443039A01261205C01A914199
:105500003605001C7141CE07400830434908C018D9
:1055100051412A46234600F02EFACDE7FFE70498D2
:1055200001224000C117121A00238B410498314612
:10553000C417381AA141EEE730B40124E4076340F0
:1055400030BC55E730B40124E407614030BC4FE77C
:105550000000E0FFF0B51FB488B00B990998002453
:1055600048400999C00F490049080991C0070B99A3
:105570000090490049080B9109990898A6460843EC
:105580001CD00B990A98084318D0099801244000B0
:10559000420D4800410D099824050003000B2043EB
:1055A00009900B980003000B20430B9050181C49E6
:1055B0004018002201901446104605E000200146E4
:1055C0000DB0F0BD032801DA034600E003239C463A
:1055D000C11A0AAE0AE05F0008ADED5B4F00F75B51
:1055E0007D430027AA187C41491C5B1E6145F2DD02
:1055F000410004AB5A522104120C0A43240C401CF3
:105600000828DFDB01980290009970460191009014
:10561000059B049A0799069800F0BAF9D0E70000B4
:105620000DFCFFFFF0B50C465C4085B0E40FE407CD
:1056300003944C0000266408590094464908024629
:105640000296224321D062460A431ED06200570DC3
:105650004A000E032303550D012402462C4924055C
:10566000781B1B0B360B40182343264361460090E2
:105670001C46501AB44103D30098401C009002E02D
:10568000921800985B41002803DA0020014605B01B
:10569000F0BD0020012109050746864611E0644659
:1056A0001D46141BB54106D36546521BB3417446D3
:1056B00007430C43A646CD074008490828439218E3
:1056C0005B4105460D43EAD11046184313D06046AE
:1056D000194650407140084306D06046101AB34145
:1056E00006D20122002306E000220123DB0702E0AC
:1056F0000122D2435310009874460105381C6141C1
:10570000029C039D0019694100F035F9BFE70000D4
:10571000FD0300000EB505490291002100910A46E3
:105720000B46019100F034F903B000BD33040000D2
:10573000410040020122400AD205090E80187F294B
:1057400001DA00207047962903DC9622511AC840DE
:1057500070479639884070474A0009030123090BB6
:105760001B051943094B10B5520D9A4201DA00206E
:1057700010BD064B34339A4203DC9A1A00F05EF8EF
:1057800010BD03495118884010BD0000FF03000000
:10579000CDFBFFFFC20FD207400040080BD0C10D68
:1057A0000723DB01C91840020905400A1143C2085A
:1057B00040071143704700200146704710B500298B
:1057C00004DB0124E40740428C412146002B04DB2A
:1057D0001C460123DB075242A341994200D190426B
:1057E00010BD0000CB0FDB07490010B54908024689
:1057F0000A4307D00A0D07240903E401090B121B11
:10580000002A01DC002010BDC900440F0C43C10078
:10581000E018D205801800F06DF810BD10B5202AF0
:1058200004DB0146203A9140002010BD9140202326
:105830009C1A0346E3401943904010BD10B5202A3E
:1058400004DB0846203AD040002110BD0B46D3406F
:10585000D0402024A21A91400843194610BD10B52B
:10586000202A06DBCB170846203A1041C1170B430C
:1058700006E00B461341D0402024A21A9140084371
:10588000194610BDF7B5009C0F4600262578641C0C
:10589000002D05D000F000F90068405DC007F5D18B
:1058A0002B2D02D02D2D18D0641E39462046029A89
:1058B00000F0F6F8002F04D03968A14201D1009918
:1058C00039607105022400290BDA4042002803DD0B
:1058D00006F0DEFE0460A007FEBD01208002064344
:1058E000E3E70028F8DA06F0D3FE04600048FEBDC6
:1058F000FFFFFF7F002904DA401C490001D1400866
:105900004000704770B40024050C05D11024000439
:1059100002D1002921D01124050E01D10002083442
:10592000050F01D10001241D850F01D18000A41CA9
:10593000002801DB4000641C002908D020252E1B14
:105940000D46F540A14000D001212943084301063E
:105950001B1B000ADB1D02D5002070BC7047DB0555
:10596000181880180029F8DA401C4900F5D170BCDD
:1059700040084000704710B5002B08DA0024401C96
:10598000614192185B411A4301D14008400010BDAB
:10599000F0B51FB482B005460C0003D0084606F0EF
:1059A0002BFE02E006F028FE203002460090214641
:1059B0002846FFF733FF049B059A04460F46184319
:1059C0001143084314D0184610431BD000984021BF
:1059D0000A1A18460599FFF731FF05460E46009A48
:1059E00005990498FFF71AFF084305D0012004E049
:1059F0002046394607B0F0BD0020C11705430E43CD
:105A00002C43374300990E986305401A7905E40A40
:105A100000220C43FD0A0A3002D500200146E9E7C6
:105A20000105101969410C9C0D9D00196941FFF792
:105A3000A2FFDFE74A0009030123090B1B051943F5
:105A40000A4B10B5520D9A4202DA0020014610BDF1
:105A5000064B34339A4203DC9A1AFFF7EFFE10BD6F
:105A6000034BD218FFF7DAFE10BD0000FF03000061
:105A7000CDFBFFFF064C0125064E05E0E36807CC91
:105A80002B430C3C98471034B442F7D3FFF71CFB70
:105A900034D6000854D600080048704794D4000853
:105AA000F7B582B0029C00272078641C1546019748
:105AB000302802D0002D15D015E020780127641C75
:105AC000782804D0582802D0002D09D00BE0002DF2
:105AD00001D0102D07D1002710252078641C02E08A
:105AE000082500E00A250026009610E0009901270D
:105AF00069430818020C294680B2714300908E1841
:105B00003804864201D3012001902078641C294684
:105B100000F019F80028E9DA0398002805D0002FD2
:105B200001D0641E00E0029C04600198002806D0A9
:105B300006F0AEFD02210160C81E05B0F0BD00995F
:105B400030040843F9E73A2800D2303820230246CF
:105B50009A43412A01D310463738884201D30020A6
:105B6000C043704770B58C180578401C6B075B0FFD
:105B700001D10378401C2A1106D10278401C03E0B1
:105B800006780E70401C491C5B1EF9D12B0705D40A
:105B90000023521E0DD40B70491CFAE70378401CF9
:105BA000CB1A921C03E01D780D70491C5B1C521E21
:105BB000F9D5A142D8D3002070BD70B50446206845
:105BC0008168490727D5816810254907002905DA2A
:105BD0008168890702D481682943816001F022FB32
:105BE000064620688068400715D501F01BFB801B26
:105BF0000A280CD920688068400708D5606D2843C2
:105C00006065A06D01210843A065012070BD20687A
:105C100080684007E9D4002070BD000038B5044614
:105C2000094808490068FFF763FA6043009000984C
:105C3000002805D00098401E009000980028F9D157
:105C400038BD000040420F0008010020F8B50446AE
:105C5000206881688907890F012934D10168C90743
:105C600031D081680522114010250126012907D075
:105C7000606D28436065A06D3043A0650120F8BDCC
:105C8000816802221143816021680320086001F0CD
:105C9000C9FA074620688068C00714D001F0C2FA2C
:105CA000C01B0A280BD920688068C00707D0606D28
:105CB00028436065A06D3043A0650120F8BD2068D1
:105CC0008068C007EAD10020F8BD0000F8B504469E
:105CD000206881688907890F012902D10168C907F5
:105CE00033D181681A4A102611400125002907D0B6
:105CF000606D30436065A06D2843A0650120F8BD4C
:105D00008168294381600120FFF788FF01F08AFA4A
:105D1000074620680068C043C00716D001F082FA29
:105D2000C01B0A280CD920680068C043C00707D0F0
:105D3000606D30436065A06D2843A0650120F8BD0B
:105D400020680068C043C007E8D10020F8BD00000B
:105D50001700008010B50E4801F064F800F05CFAFE
:105D600005F020F900F0CAFB0A480B49808C086056
:105D70000A4C0020E06000F0EBF8094800F042FD1A
:105D800000F062F9207003F0F1FF002010BD000068
:105D9000B80B000074060020280000203800002006
:105DA000F1640008F8B503F091FA03F043FE00F047
:105DB000D1FC04F01DF8524D524C2878A1780843CC
:105DC00001D104F0B5F903F0FBFF012801D103F084
:105DD00035FE03F0F5FF012811D100F0B5FB0128D5
:105DE0000DD1207900280AD103F05AFE002806D1EF
:105DF0006079002803D144480078002802D0287830
:105E0000012801D104F0C8FB2878404F0126002565
:105E1000002806D103F0D4FF012802D1A078002881
:105E200010D004F099FBA571267236481430818891
:105E3000006801F0E9F9012852D0334800780028C1
:105E400058D05AE03248007800283FD0A079002886
:105E500004D0012826D002283BD133E03868E1681D
:105E6000401A2C49898C884202D8207A012830D1E6
:105E70002572657028A003F0EFF804F079FBA67195
:105E80003868E06003F00CFE002822D1254928463E
:105E90000D6025490B6825490A682549096804F001
:105EA00045FF16E03868E168401A3C2811D9E670D1
:105EB000267120A003F0D0F804F04EFBA5713868DD
:105EC000E06006E0E67026711DA0F3E704F044FBF5
:105ED000A5710D4800780128A7D100F067F9A4E763
:105EE0003878C00702D000F061F901E000F040F915
:105EF000667102E000F03CF965710020F8BD000019
:105F000030000020380000209900002028000020E8
:105F10000200002074060020475053204F4E0D0A07
:105F20000000000024000020180000201C000020B9
:105F300020000020475053204F46460D0A00000025
:105F400047505320535543434553530D0A00000017
:105F500010B5012007F0B4F80A4C1328A0700AD03D
:105F6000E01C03F0D7FDE078A070332806D0064986
:105F70000020C88710BD07F0DBF810BD03F09CFDC2
:105F800010BD0000D80000207406002010B500F0FD
:105F900003F8002010BD000070B50524FF2224077F
:105FA00001322146012004F0EFFA1749002006F0E3
:105FB00073F91649022006F06FF91549012006F021
:105FC0006BF9144D012292032946002003F002FFD1
:105FD00004222946012003F0FDFE01221203294676
:105FE000022003F0F7FE10222146002000F0AAFB59
:105FF0000021094800F0FCF80122D20221460120CC
:1060000000F070F8002070BDCC0400205405002082
:1060100044040020000400503406002010B5002481
:10602000084800F02DFE611E064800F0C1FD002862
:1060300003D1044800F096FC0446024800F050FEEC
:10604000204610BDB803002070B5002400F026F8EB
:106050000D4E0546B04215DB00200C4A0C4B0146A4
:10606000FFF7ACFB01D264240CE031462846FFF771
:106070002FF90849FFF771F90749FFF731F9FFF7E1
:1060800057FB0446204670BD33335340CDCCCCCCB7
:10609000CCCC10406666663F0000C84210B500F0E8
:1060A00017F8642000F0BEFEFFF7B8FF00F048F8D4
:1060B000044600F003F8204610BD000010B5034868
:1060C00001228189806801F0A6F810BDDC11002052
:1060D00010B5034800228189806801F09CF810BD4A
:1060E000DC110020022802D30020C0437047C30007
:1060F0000248C1501818828000207047DC1100202F
:1061000010B50C4C206B002812D16169A06A401AAE
:106110003C280DD3084900200870FFF795FFC1B255
:1061200006486429017001D964210170A06A606188
:1061300010BD0000000000203A00002038000020C0
:1061400010B5FFF7E7FA0022064BFFF76BFA064A95
:10615000064BFFF7FFF9FFF745FB0121FFF73BF97E
:1061600010BD000000FEAF406666666666660A40C7
:1061700010B50D4C002320460068616802680029B4
:106180000BD004290BD008290BD0136402F066FA57
:10619000206802F0D5F8002010BD5363F6E7936342
:1061A000F4E7D363F2E700008000002010B50F4C45
:1061B000206802F095F803CC083C02F005FA61680B
:1061C0003C20002908D004290AD008292168096840
:1061D0000AD00864002010BD216809684863F9E707
:1061E000216809688863F5E7C863F3E78000002049
:1061F000014A03C2002070478000002010B5002330
:106200001A4603E0845CE3189BB2521C8A42F9D31D
:10621000D84380B210BD000000B587B001216846A8
:106220004170022101700D480190C8010290800068
:106230000490402005906946002005F079FF07484A
:106240000749203801610749C16107498161074950
:106250004161074802F030FF07B000BDDC100020AC
:106260008162000875620008B1620008BF62000820
:106270003C0B002010B50146002005F019FF10BDB1
:106280000FB400B5FFB082B0012183AB490268466C
:10629000829A06F09BF96846FEF7A8FF0246694617
:1062A000002006F05DF87FB002B008BC04B01847CB
:1062B00001B501226946002006F052F808BD10B56C
:1062C0000446FEF793FF02462146002006F048F8F8
:1062D00010BD30B4446C1C252C400125A540046C35
:1062E0006560046863608368102B05D0036899605B
:1062F0000068C26030BC704703689A600068C16083
:1063000030BC704708B503E06846007806F0D6F860
:106310006946002005F0CCFE0028F5D008BD10B578
:10632000012000F0ABFE022000F0A8FE10BD10B569
:10633000202000F0A3FE802000F0A0FE10BD000091
:1063400010B4084900234B6107494A684C152243A1
:106350004A604A68082422434A60C009C0010360B9
:1063600010BC704788290020002002407FB500251E
:106370000C460646039500F0D3FDE009029003A900
:1063800001960095684600F05FFD002804D000F0FB
:106390009BFD002004B070BD00F096FD0120F9E7E0
:1063A00010B5002302E0C45CCC545B1C9342FAD3CA
:1063B00010BD000010B40020204A9169CB0520498F
:1063C00004D54869022318434861901593699B05D9
:1063D00005D54B69012423434B616302184393693C
:1063E0005B0505D54B69082423434B61E301184342
:1063F00093691B0505D54B69042423434B61630254
:10640000184393699B0405D54B69102423434B61C2
:106410006302184393699B0304D54C6920231C43F2
:106420004C6118439369DB0305D54B694024234332
:106430004B61A1020843906110BC704700200240EC
:106440008829002070B5044600F0ECFE0546194E80
:10645000B069C0070DD0601C08D0002C04D000F03B
:10646000E1FE401BA04201D9032070BDB069C00706
:10647000F1D1B069800701D50220B061B069C005D3
:1064800011D4B06980050ED4B06940050BD4B06951
:10649000000508D4B069800405D4B069800302D433
:1064A000B069C00303D5FFF785FF012070BD002050
:1064B00070BD000000200240F8B5174600260546D2
:1064C0000C4600F02DFD09E029460220226800F06C
:1064D00009FD002804D1241D2D1D361DBE42F3D315
:1064E00000F0F2FCBE4201D20020F8BD0120F8BD50
:1064F00001490220887170473800002000B587B03C
:10650000012069464870022008700C49019141023F
:1065100002910B49039105214902049105906946B6
:1065200005F006FE8821074802F07AFF05200122C7
:106530001021000700F06FFE07B000BD6C120020B4
:106540006C1600207C20002003480078002801D031
:1065500000207047012070478C000020F0B593B0F8
:106560000E460546282108A8FEF721FE03AA009240
:106570002846314601AB4FA202F083FF0027FF43BC
:1065800002281AD10499039802F06BFFC2B2019855
:106590000178012003E0019B1B5C5940401C029BD9
:1065A0008342F8D8914208D1002406AB44A2314678
:1065B000284602F066FF0F2802D0384613B0F0BD1F
:1065C000A819801E0470447049482B460278494837
:1065D0004188049202910394059447498088097880
:1065E00001910090FF2145A201314B4803F03CF896
:1065F000074680214948FEF7DAFD3A4646494748B2
:10660000FEF7BCFD464D474EAF7006983946007800
:10661000302841482AD002F03FFD6868002846D063
:1066200041A002F019FD6B683A463B4900209847AB
:106630006878002803D0FF2030606C7002E00120F1
:106640003460687037483C4D3C4E3D4F02682B68C3
:106650003168386804F06AFB642000F0E3FB3148DD
:10666000224604602B68316838681EE002F014FD91
:106670006878002804D0FF20000230606C7002E0CF
:106680000120346068702C4D2C4F2D482B683268E7
:106690003968006804F04AFB642000F0C3FB3460F2
:1066A000274822462B683968006804F03FFB002029
:1066B00084E700002425702A25700D0A00000000E0
:1066C00024252A2C252A2C252A2C252A2C252A2C3F
:1066D000252A2C25702C252A2C252A2C252A2C25E8
:1066E0002A2C252A2C252A2C252A2C252A2A00006A
:1066F0003D000020740600203800002025732C2562
:10670000582C253032782C25782C25642C25782C93
:106710002564250D0A00000004210020EC11002052
:106720008C0000201C0000204C4F52412046414666
:1067300041464146410D0A0018000020200000207B
:1067400024000020C3000248C150181882807047FE
:106750006C20002008B500206946087003E06846F8
:10676000007800F013F86946022005F0A1FC00282B
:10677000F5D008BD01490020087070478C0000204A
:1067800001490120087070478C00002070B51A4D37
:1067900000262C462B78611C8034002B08D0224622
:1067A0005268022B0CD0032B09D10A2813D021E008
:1067B000242804D102222A7070540120606070BD28
:1067C00050546168491C61607E2913D20D28F6D1AE
:1067D0000320287070BD50546068401C60604654AF
:1067E00006A1681CFEF7EEFC002803D0681C616857
:1067F000FFF7B4FE2E7070BD7C2000204747412C6F
:106800000000000001494860704700008C00002033
:10681000F8B50C4605464035297C01290DD00121EB
:10682000297401688A68520709D5416D20221143F5
:106830004165002028740120F8BD0220F8BD194BE5
:106840006268D8054710184E9A4215D08A6A2368A4
:106850005B035B0B1A438A622168490305D5B16863
:106860000143B1600A20FFF7D9F92068800315D5EC
:10687000B0683843B06011E08A6A23685B035B0B41
:106880009A438A622168490302D5B1688143B160A5
:106890002068800302D5B068B843B0600020287437
:1068A000F8BD0000011000000027014070B504464B
:1068B000002C0AD0606D0221084360652046FFF776
:1068C0007CF90546280002D009E0012070BD204671
:1068D000FFF7BCF90546012D01D0012060650026B7
:1068E000012D32D0206841681A4A11404160216868
:1068F000D0430860206881680122120791438160BB
:106900002068C168144A1140C16020680169134AB7
:106910001140016120684169C908C90041612068CE
:10692000016A0F4A1140016220688030416BC90939
:10693000C901416320688030416BC909C9014163C5
:10694000204600F0F9F8A6656665403426742846AE
:1069500070BD000060F7FFFF00023E8302FCFF3FB6
:1069600000F000F00068006C7047000070B504464D
:10697000002C06D0606D264600254036002802D047
:1069800006E0012070BDA5653574204600F0E8F8EA
:10699000606DC00603D420688168490706D5606D24
:1069A0001021084360653574012070BD616DFF22C0
:1069B0000132914302221143616581685C4A890773
:1069C000890F012902D10168C9072BD1032361680E
:1069D0009B07994205D05B42994202D05B009942E5
:1069E00009D101698900890801612068016963682A
:1069F000194301610CE0016989008908016190680F
:106A00000F21890488439060906861680843906012
:106A10002068C16818239943C1602068C168A368D1
:106A20001943C160906801214906884390609068CD
:106A3000A18E49060843906020688168C90004D48B
:106A4000816801221207114381602068C168394AB8
:106A50001140C1602069E268022825D0002002436D
:106A6000204620300178037B49035B0019430A4329
:106A7000216B0A43A16989030A43E169C9030A43F7
:106A80002168CB681A43CA60616A0A46FF3AC23A73
:106A900005D0A26A11432268D3681943D1604278B5
:106AA0000121012A02D00BE00420D8E70078002859
:106AB00023D0606D202210436065A06D0843A0655F
:106AC000E06B012820D020680169C90703D0016963
:106AD00049084900016120684169C908C90041614C
:106AE00020684169A26B11434161A565606D800812
:106AF0008000401C6065002070BD2068C2680123D2
:106B00001B041A43C260DBE720680269FF239B0075
:106B10009A43026120680269236CA66C1A43636C75
:106B200033431A430261206802690A430261D2E7D3
:106B3000002701401902FEFF10B50068064988428F
:106B400009D10648416B421591434163052002215A
:106B5000000700F015FA10BD0024014000100240AB
:106B600010B586B0044614216846FEF720FB0E4996
:106B70002068884216D10D48416B4215114341638C
:106B8000C16A01221143C162C06A69461040059082
:106B900002200090032001900020029005200007B1
:106BA00000F078FA06B010BD002401400010024049
:106BB000F8B504460E4627466069403708280BD0D2
:106BC0002068C068C00709D0606D20210843606557
:106BD000002038740120F8BD082500E00C2500F0E5
:106BE00021FB009020680068284219D1701C13D046
:106BF000002E05D000F016FB0099401AB0420BD9C8
:106C000020680068284207D1606D04210843606550
:106C1000002038740320F8BD206800682842E5D0C1
:106C2000606D01214902084360652068C16809055B
:106C30008A0F0C21002A1BD12022125D002A17D1B5
:106C40000268120714D5826801235207002A08DB64
:106C500042688A434260606D1A029043184360653F
:106C600006E0606D202210436065A06D1843A065AA
:106C7000A069002801D1206801600020F8BD000053
:106C800070B50446002021688968490723D4254649
:106C90004035297C01291CD001212974E169012991
:106CA00002D02046FFF712F8002811D1616D0B4A7F
:106CB0001140FF220132114361650021A165297451
:106CC00022681C21116021688A6804231A438A60A3
:106CD00070BD022070BD022070BD0000FEF1FFFFFC
:106CE00070B5044625464035287C012807D001268A
:106CF0002E742046FEF761FF002802D00CE002202F
:106D000070BD2046FEF7A2FF002805D1616DFF226D
:106D100001329143314361650021297470BD30B463
:106D2000014620314A790023022A05D00422C26399
:106D30000B7130BC01207047026814680E25AC430B
:106D4000146002681468640864001460446C1C22B7
:106D5000144001252A46006CA24042604D710B711F
:106D600030BC1846704770B50024014620314A797E
:106D7000022A03D00421C163012418E002681368C9
:106D80000E25AB431360026813685B085B00136059
:106D9000436C1C22134001252A469A40036C5A601A
:106DA0004D7100220A71816B002900D0884720466E
:106DB00070BDF8B504468C46002520462030017988
:106DC000012909D00126067147790021012F05D03C
:106DD000017102252846F8BD0220F8BD022747713F
:106DE000E163206801684908490001606146204666
:106DF000FFF76FFA206B002805D0206801680E228B
:106E00001143016009E02068016804229143016098
:106E1000206801680A22114301602068016831433B
:106E20000160D7E770B5044600F0FCF90546601C28
:106E300002D004480078241800F0F4F9401BA04266
:106E4000FAD370BDFC000020F8B505460E461B4F76
:106E5000387C012808D0012038741948FFF7F2FA6D
:106E60000146080002D025E00220F8BD0020C04302
:106E700030606C68A868C0010019A0421AD9204689
:106E8000FFF75EFA0E48FFF7DDFA01460D4842684B
:106E900008239A434260426843159A43426000299E
:106EA00001D0346006E08034A8686A68C0018018A8
:106EB000A042E4D8002038740846F8BD8829002094
:106EC00050C30000002002400548416802221143DF
:106ED0004160416801221143416000207047000079
:106EE00000200240F8B50E4617460B4C207C0128C6
:106EF00008D0012020740948FFF7A4FA00250028D3
:106F000002D006E00220F8BD656137600348FFF754
:106F100099FA2574F8BD00008829002050C30000AC
:106F200012494868C0070DD0EFF3108072B6104ABE
:106F3000CA60104ACA6080F310884868C00701D050
:106F400001207047486880070DD5EFF3108072B6B6
:106F5000094A0A61094A0A6180F310884868800773
:106F600001D501207047002070470000002002403A
:106F7000EFCDAB8905040302BFAE9D8C161514132B
:106F8000F0B50022002961D0012393409E460B40BA
:106F9000002B57D095082E4CAD002D19AC689607E4
:106FA000360F0F27B7403C40A44605242407A042D3
:106FB00001D1002419E0274CA04201D1012414E0A2
:106FC000254CA04201D102240FE0244CA04201D163
:106FD00003240AE0224CA04201D1042405E0214C04
:106FE000A04201D1052400E00624B44064450FD13D
:106FF0001D4C26689E43266066689E436660E66870
:107000009E43E660A6689E43A660AB68BB43AB6048
:10701000046855000323AB401C430460D408A4005B
:107020002418266A5507EF0E0F25BD40AE43266291
:10703000C4689C43C46044687546AC43446084683B
:107040009C438460521C0B46D3409DD1F0BD000090
:10705000000001400004005000080050000C0050E7
:1070600000100050001C005000040140202802D1F4
:1070700001490020086070472C00002010B5044929
:107080004A69024202D04861FFF7F0FF10BD0000DC
:1070900000040140F0B400220B68002B6FD00127E0
:1070A0000B6897403B40002B6AD00C79A407A40FD3
:1070B000012C01D0022C10D1856854000326A64073
:1070C000B543CE68A6402E4386604468BC430D7924
:1070D000ED06ED0F9540254345600C79E443A40788
:1070E00008D0C56854000326A640B5438E68A64064
:1070F0002E43C6600C79A407A40F022C0CD1D4082F
:10710000A40027183D6A5407E40E0F26A640B54395
:107110000E69A6402E433E62056854000326A64031
:10712000B5430E79B607B60FA6402E4306604C68ED
:10713000A403A40F50D02C4C656B01263543656326
:1071400095082A4CAD002F19BD689407240F0F260F
:10715000A640B54305263607B04201D100261BE004
:10716000234EB04201D1012616E0224EB04201D199
:10717000022611E0204EB04203D103260CE030E09D
:107180002AE01E4EB04201D1042605E01C4EB0425A
:1071900001D1052600E00626A6402E43BE60194D0B
:1071A000AC689C434E68F60200D51C43AC60EC68AA
:1071B0009C434E68B60200D51C43EC606C689C434F
:1071C0004E68B60300D51C436C602C689C434E6827
:1071D000F60300D51C432C60521C0B68D34000D032
:1071E0005DE7F0BC70470000001002400000014065
:1071F0000004005000080050000C00500010005027
:10720000001C0050000401400069084201D0012028
:10721000704700207047002A01D081617047816269
:10722000704700000148806870470000FC000020A3
:1072300004494A6B01231A434A6303494A680243DB
:107240004A60704700100240000001400248816817
:107250000278891881607047FC00002010B5002476
:1072600007480168402211430160032000F00AF83A
:10727000002801D0012401E000F08EF9204610BD65
:107280000020024070B504460E4D7D202978C000D4
:10729000FDF72EFF01460C480068FDF729FF00F0BE
:1072A0006FFF002801D0012070BD042C07D20022FE
:1072B0002146501E00F098F96C60002070BD01203E
:1072C00070BD0000FC0000200801002070477047DE
:1072D00010B51548816A491C8162C26A1349521C63
:1072E000C2624B8F0021934202D20122026300E06E
:1072F00001630F4B1878012807D10E480268521C11
:107300000260022A01D3016019700B4A107801282B
:1073100009D10A4B1878401E0006000E187002D1E1
:107320001170FEF725FF10BD00000020740600203C
:107330003C0000205C000020990000209800002004
:107340007047704770472030807B704710B5044607
:1073500020680168C943C90708D18168C943C907C2
:1073600004D1012141602046FFF7B2FF2068016887
:10737000C943890708D48168C943890704D4022115
:1073800041602046FFF7A2FF20680168C943490712
:1073900008D48168C943490704D4042141602046C8
:1073A00000F0F8F820680168C943090708D481682B
:1073B000C943090704D4082141602046FFF7C0FFF4
:1073C00020680168C943C90608D48168C943C90651
:1073D00004D4102141602046FFF779FF206801683E
:1073E000C943890608D48168C943890604D4202189
:1073F00041602046FFF7A6FF20680168C94349069F
:1074000008D48168C943490604D44021416020461C
:10741000FFF797FF10BD0000F8B50446002C06D01A
:10742000606825462035A87B002802D006E00120B0
:10743000F8BD00206873204600F046F80220A873CB
:1074400020688446C0686168012904D00122A36ACB
:10745000D205934201D11E229043184B62699A4291
:1074600001D0174B1840174B1840A368676A266A6B
:107470000B433E431E43A36A1E433043002903D1FE
:107480002769E6693E433043012903D00121C9053C
:107490008B4203D12369E1681943084307498A42B3
:1074A00005D0A1690A43E1690143104608436146DA
:1074B000C8600120A8730020F8BD0000FFFF000095
:1074C0003F1FFFFFFEF119FF10B500680849884211
:1074D0000CD10848816BC20411438163002211461C
:1074E0000D2000F081F80D2000F072F810BD0000B2
:1074F000007C004000100240F8B504461646022207
:10750000204620300546827321480268C3041A438E
:1075100002602068C2689B121A43C2602068026938
:1075200001273A430261226810205060206881617F
:107530001021204602F0BCFB032822D0216808203D
:107540004860206846610821204602F0B1FB03280C
:1075500019D0204602F032FB2046FFF7F4FE032844
:1075600013D02068816839438160206801693943FC
:10757000016120680169042211430161AF73002099
:10758000F8BD0320F8BD0320F8BD0320F8BD0000BE
:1075900000040140704700000448416B0122114380
:1075A0004163816B02041143816370470010024004
:1075B000002809DBC106C90E012088400349086084
:1075C000BFF34F8FBFF36F8F7047000080E100E083
:1075D000002805DBC106C90E01208840014908606A
:1075E0007047000000E100E08207D30EFF229A40BE
:1075F0008907090E9940002808DB830809489B0089
:107600001818036893430B43036070470007000F8B
:107610000838830804489B001818C36993430B4338
:10762000C361704700E400E000ED00E0024801683B
:10763000821511430160704700700040F0B4164E8F
:10764000326875152A40154B1B6ADB07DB0F002AD1
:1076500004D0002B02D03468AC4334603468A408F2
:10766000A400044334600E4F3C69042004433C6191
:1076700001290ED040BF20BF20BF39698143396145
:10768000002A04D0002B02D0306828433060F0BCC0
:10769000704730BFF1E7000000700040000001407B
:1076A00000ED00E0F8B50446002620785E4D800627
:1076B0007DD55E48806BC00005D45C48816B0204B8
:1076C0001143816301265A480168C90517D400682F
:1076D000FF210131084356490860FFF7A3FD074623
:1076E00053480068C0050AD4FFF79CFDC01B6428FE
:1076F00001D90320F8BD4E480068C005F4D54B4FB2
:10770000386803210905084062681140814208D0A9
:107710009003800F032804D13868800301D501202D
:10772000F8BD2869032109040840002824D00A4034
:10773000824221D0207880061ED5286988432A6994
:107740000121C9040A432A612A698A432A612861FE
:10775000C00511D5FFF766FD0090286980050BD4A0
:10776000FFF760FD0099411A3248814201D9032098
:10777000F8BD28698005F3D52078800611D56068AA
:107780008103890F032905D13A6809058A43084016
:1077900002433A60286903226168120411400843D9
:1077A0002861012E03D1B96B30078143B96320787A
:1077B000C00705D0E868A168800880000843E86039
:1077C0002078800705D5E8680C218843E1680843E4
:1077D000E8602078400706D5E868032189028843DD
:1077E00021690843E8602078000706D5E86803218E
:1077F0000903884361690843E8602088C00506D50D
:10780000E968032000048143A0690143E96020780E
:10781000000606D5E868032189048843E169084326
:10782000E8600020F8BD0000401002400010024057
:107830000070004088130000F8B504460D46002C87
:107840001BD076480068C007C00FA8421CD2734FF7
:1078500038684008400028433860FFF7E3FC0646DC
:107860003868C007C00FA8420ED0FFF7DBFC811BB1
:107870006B48814203D90320F8BD0120F8BD386868
:10788000C007C00FA842F0D12078664F800705D509
:10789000F868F0218843A1680843F8602078C007A1
:1078A00072D06068022808D003280BD001280ED0BF
:1078B0003968890510D40120F8BD396889030BD4D3
:1078C0000120F8BD3968890106D40120F8BD396866
:1078D000490701D40120F8BDF968890889000143EE
:1078E000F960FFF79FFC0646606802280FD0032866
:1078F00020D0012831D0F8680007800F44D0FFF76E
:1079000091FC811B464881423AD90320F8BDF868B2
:107910000007800F022837D0FFF784FC811B404806
:10792000814201D90320F8BDF8680007800F0228C2
:10793000F2D129E0F8680007800F032824D0FFF770
:1079400071FC811B3648814201D90320F8BDF868DB
:107950000007800F0328F2D116E0F8680007800FB7
:10796000012811D0FFF75EFC811B2D48814201D90F
:107970000320F8BDF8680007800F0128F2D103E06A
:10798000F8680007800FBAD124480168C907C90FF9
:10799000A9421CD9006821494008400028430860DA
:1079A000FFF740FC06461D480068C007C00FA8420C
:1079B0000DD0FFF737FC811B1948814201D9032004
:1079C000F8BD16480068C007C00FA842F1D1207862
:1079D000400706D5F868072109028843E168084393
:1079E000F8602078000707D5F8680721C9028843A6
:1079F0002169C9000843F86000F042F8F9680A4AB2
:107A00000906090F515CC840084908600848006829
:107A1000FFF738FC0028D3D1F8BD00000020024059
:107A20008813000000100240F0D300080801002075
:107A30000001002001480068704700000801002094
:107A400000B5FFF7F7FF0449C968044A4905490F23
:107A5000515CC84000BD00000010024009D400087D
:107A600000B5FFF7E7FF0449C968044A8904490FD4
:107A7000515CC84000BD00000010024009D400085D
:107A800070B5214EF2680C21104608401F498B004A
:107A900004280CD04D00082810D00C2810D0706895
:107AA0000004410F491C0120C003884070BD3068AC
:107AB000C00601D5084670BD184670BD284670BD89
:107AC0009002134C000F205C1202940F641CF268A9
:107AD000D20307D5294604F0A6FD22460023FDF770
:107AE0001DFB70BD3268D20606D504F09CFD22460F
:107AF0000023FDF713FB70BD194604F094FD2246E8
:107B00000023FDF70BFB70BD0010024000093D0093
:107B100000D40008F0B583B00446002C0FD0F84E16
:107B2000F5680C200540F768012000040740207824
:107B3000C0075BD0082D09D00C2D03D00FE0012029
:107B400003B0F0BD01200004874208D130688003F3
:107B50004CD56068002849D1012003B0F0BD012058
:107B600061680004814203D131680143316015E04E
:107B7000052301221B049204994206D13168114366
:107B8000316031680143316008E031688143316020
:107B9000316801400191306890433060606800288E
:107BA00012D0FFF73FFB0290306880031ED4FFF72E
:107BB00039FB0299401A642802D9032003B0F0BDB2
:107BC00030688003F3D511E0FFF72CFB029030689A
:107BD00080030BD5FFF726FB0299401A642802D9CF
:107BE000032003B0F0BD30688003F3D42078800711
:107BF00068D5E068810604D5326820210A433260E6
:107C000088430923042D17D00C2D01D1002F13D048
:107C1000002842D03168994301433160FFF702FBED
:107C20000746306840072FD4FFF7FCFAC01B022834
:107C300027D9032003B0F0BD3168490701D50028DA
:107C40001CD071681F221202914322691202114353
:107C500071603168994301433160FFF711FFF168AA
:107C600009060A0FA749895CC840A7490860A748C8
:107C70000068FFF707FB0028DCD123E0012003B0F8
:107C8000F0BD30684007CFD570681F2109028843D6
:107C9000216909020843706014E030684008400020
:107CA0003060FFF7BFFA0746306840070AD5FFF794
:107CB000B9FAC01B022802D9032003B0F0BD306816
:107CC0004007F4D42078C0066BD5002D15D0A069EC
:107CD000002850D03068FF21013108433060FFF7A1
:107CE000A1FA07463068800536D4FFF79BFAC01B1F
:107CF00002282ED9032003B0F0BD3068800502D5DC
:107D0000A069002822D07068072149038843216AAE
:107D1000084370607068217F0002000A090608436A
:107D20007060206A410B491C0120C0038840F16843
:107D300009060A0F7349895CC84073490860734893
:107D40000068FFF79FFA0028D5D12AE0012003B090
:107D5000F0BD30688005C8D57068072149038843A5
:107D6000216A084370607068217F0002000A0906DA
:107D70000843706015E03168FF20013081433160B5
:107D8000FFF750FA0746306880050AD5FFF74AFA30
:107D9000C01B022802D9032003B0F0BD3068800563
:107DA000F4D420785A4F00072FD56069002816D0E8
:107DB0003869012108433861FFF734FA02903869C5
:107DC000800722D4FFF72EFA0299401A022802D91E
:107DD000032003B0F0BD38698007F3D515E038699A
:107DE000400840003861FFF71DFA029038698007AB
:107DF0000BD5FFF717FA0299401A022802D903207F
:107E000003B0F0BD38698007F3D42078400775D5FA
:107E100000200190B06BC00006D4B06B01210907AF
:107E20000843B063012001903A480168C90519D49C
:107E30000068FF210131084336490860FFF7F2F975
:107E4000029034480068C0050CD4FFF7EBF90299A2
:107E5000401A642802D9032003B0F0BD2D48006801
:107E6000C005F2D5FF20A2680130824203D13969F2
:107E7000014339611BE001218902002A0AD0052350
:107E80001B029A420DD13A690A433A6139690143AA
:107E900039610CE03A6982433A6138698843386154
:107EA00005E03A6982433A61386988433861A068DD
:107EB000002813D0FFF7B6F902903869800530D456
:107EC000FFF7B0F90299411A1348814202D9032001
:107ED00003B0F0BD38698005F2D522E0FFF7A2F9C2
:107EE0000290386980051CD5FFF79CF90299411A68
:107EF0000948814212D9032003B0F0BD19E0000007
:107F000000100240F0D3000808010020000100200A
:107F1000401002400070004088130000386980055E
:107F2000E2D40198012804D1B06B012109078843EC
:107F3000B063606A002864D00C2D49D001252D065D
:107F400002280FD03068A8433060FFF76BF9044671
:107F50003068800155D5FFF765F9001B022833D939
:107F60000320C9E73068A8433060FFF75BF9074694
:107F70003068800109D5FFF755F9C01B022801D9E7
:107F80000320B9E730688001F5D4E16AA06AF2689D
:107F90000843216BFD231B049A4311430843F060FF
:107FA000306828433060FFF73DF9044630688001AF
:107FB00027D4FFF737F9001B022801D903209BE7DC
:107FC00030688001F5D51CE030688001C3D418E02A
:107FD000012814D0F06801210904A26A01409142ED
:107FE0000BD10F218904E26A0140914205D103219E
:107FF00089050840216B884203D001207CE70120DD
:108000007AE7002078E70000024801690222114364
:108010000161704700E000E070B50446002C10D00C
:10802000022025464035687420680168402291434B
:108030000160204600F064F80020606568742874D0
:1080400070BD012070BDF8B50446002C0ED0FF278E
:10805000606A0537002600280AD026616661A6629C
:1080600025464035687C002807D00AE00120F8BD8D
:108070006068B842F3D0E661F1E72E74204600F064
:1080800053F8022169742068026840239A43026011
:108090002123A26860689B021A4038401043E368BD
:1080A0008A021340184323690B40217D1843C907F6
:1080B000C90F0843A169931019400843E1693823A7
:1080C00019400843216A802319400843A16A93009C
:1080D0001940084321680860A0690421000C084089
:1080E000616A102319400843216848602068C1690B
:1080F0009143C1616665012068740020F8BD0000ED
:1081000010B500680649884209D10648416B8214BF
:10811000914341630520E0210007FEF731FF10BDC8
:10812000003001400010024010B586B00446142112
:108130006846FDF73CF810492068884219D10F487D
:10814000416B821411434163C16A01221143C16230
:10815000C06A002110400590E020009002200190AC
:108160000320039002910491052069460007FEF761
:1081700091FF06B010BD0000003001400010024029
:1081800010B40B49401E884202D910BC0120704730
:108190000849486108480723C2691202120A4C04C0
:1081A0002243C261002088610B6110BC704700004F
:1081B000FFFFFF0000E000E004ED00E0024801697D
:1081C000022291430161704700E000E0F0B40246F2
:1081D0002032137E012B22D00126167602235376FD
:1081E00003685D689C687027BD430F682F435F601C
:1081F0000068B307984208D00A4B984205D00A4B52
:10820000984202D0094B984204D180239C4349688C
:1082100021438160567600201076F0BC7047F0BC98
:108220000220704700040040000801400014014093
:1082300010B5022104462034617601680A6A094BB0
:108240001A4203D10A68520852000A6000F02CF862
:108250000020A077A076E0762077607760762076A1
:1082600010BD00001111000070B50546002D05D0AD
:108270002C462034607E002802D006E0012070BD2C
:1082800000202076284600F01DF802206076291D87
:10829000286803F08BF80120A077A076E07620779D
:1082A00060776076002070BD00680449884204D180
:1082B0000348416B04229143416370470008014029
:1082C0000010024000680449884204D10348416B11
:1082D000042211434163704700080140001002402E
:1082E000014620314A7E012A01D001207047022236
:1082F0004A760168CB6801221343CB60006891077E
:10830000884208D00B49884205D00B49884202D0E8
:108310000A49884208D181684907490F062906D0D1
:1083200001681143016002E001681143016000200F
:1083300070470000000400400008014000140140A4
:108340000168CA6852085200CA6001680A6A064B8E
:108350001A4203D10A68520852000A6001212030F3
:10836000417600207047000011110000F8B5044666
:10837000002625462035287E012817D001202876A2
:1083800002206876206882687727BA43FF231B02A1
:108390009A4382600868502838D00EDC202853D0D9
:1083A00006DC002850D010281ED14DE00220F8BD78
:1083B000302849D0402817D13CE0602830D07028C0
:1083C00019D001221203801A0FD090420CD1CB6831
:1083D0004A688968206803F02BF8206881680122C8
:1083E00092031143816000E001260120687600209D
:1083F00028763046F8BDCB684A688968206803F063
:1084000017F82068816839438160EEE7CA684968D7
:10841000206803F092F85021206803F015F8E4E793
:10842000CA684968206803F09AF86021206803F060
:108430000BF8DAE7CA684968206803F07EF8402143
:10844000206803F001F8D0E722680146104602F0E8
:10845000FBFFCAE710B586B0044614216846FCF756
:10846000A6FE0D492068884213D10C48C26A022139
:108470000A43C262C06A0191084005900803009057
:108480000020029003900620049069460448FEF7FD
:1084900001FE06B010BD00000008014000100240BF
:1084A00000040050F8B504460D4600272646203645
:1084B000307E01280ED001203076002A0CD0042A0C
:1084C0001ED0082A33D00C2A45D001270020307650
:1084D0003846F8BD0220F8BD2946206802F0BCFFEE
:1084E0002068816908221143816120688169042222
:1084F0009143816120688169EA6811438161E5E700
:108500002946206802F0C1FF206882690121C90262
:108510000A4382612068816901229202914381614C
:1085200020688169EA68120211438161CEE7294619
:10853000206802F0C7FF2068C16908221143C161A9
:108540002068C16904229143C1612068C169EA6859
:108550001143C161BAE72946206802F0CFFF2068C5
:10856000C1690122D2021143C1612068C26901219F
:1085700089028A43C2612068C169EA681202114314
:10858000C161A3E770B50546002D05D02C46203407
:10859000607E002802D006E0012070BD0020207619
:1085A000284600F00FF802206076291D286802F0A6
:1085B000FDFE0120A077A076E076207760776076D8
:1085C000002070BD7047000070B505462C46203471
:1085D000002908D0042908D0082908D0627F012A80
:1085E00007D0012070BDA27EF9E7E27EF7E7227F87
:1085F000F5E70220002920D0042920D0082920D026
:1086000060770122286802F005FF012128688907A8
:108610000122884208D00E49884205D00D4988427F
:1086200002D00D4988420ED181684907490F0629B9
:108630000CD001681143016008E0A076E1E7E07624
:10864000DFE72077DDE7016811430160002070BD9E
:1086500000040040000801400014014070B50446C9
:108660000D4600222946206802F0D4FE2068016AE7
:108670000B4A114203D101684908490001600120F9
:108680002034002D06D0042D06D0082D06D06077AA
:10869000002070BDA076FBE7E076F9E72077F7E7EA
:1086A000111100007047704770B50446002C1BD0B4
:1086B0002420E067206801684908490001602068BB
:1086C000002505602068456020688560204600F030
:1086D0009BF9204680304560E56705602566656644
:1086E00060342576002070BD012070BD10B503F008
:1086F000E9FD10BDF8B504462268D0691168936899
:10870000A24D06462E40002E09D1850607D58D06BE
:1087100005D5A16E002901D020468847F8BD254621
:108720008035002E7FD09A4FDE07F60F0F4037437B
:1087300079D0C70706D0CF0504D5012717626A682C
:108740003A436A60820708D5DA0706D02768022212
:108750003A626A6804273A436A60420708D5DA0732
:1087600006D0236804221A626A6802231A436A60E8
:10877000020709D520220A40324305D02368082287
:108780001A626B6813436B60020509D54A0107D56D
:1087900001222368D2021A626A6820231A436A609F
:1087A0006A68002ABAD0800606D5880604D5A16E6C
:1087B000002901D0204688476868216889684906F1
:1087C00002D42821084228D0204603F073F82068FC
:1087D000816849061DD5EFF31081012282F31088CC
:1087E000836840229343836081F31088606F002880
:1087F0000BD068498163606FFEF7B5FA00288DD011
:10880000606F816B8847F8BD0DE02046FFF76EFF73
:10881000F8BD2046FFF76AFFF8BD2046FFF766FF68
:1088200000206860F8BD266E012E7DD1C6067BD57E
:10883000CE0679D510231362206881682646490642
:10884000403600294CDA626F1168496889B2002904
:10885000E8D0378B8F42E5D97183116809688906A2
:1088600034D4EFF31081012282F3108802681F01D3
:10887000BA43026081F31088EFF31081012080F386
:1088800010882068826852085200826081F3108844
:10889000EFF31081012080F3108820688268402760
:1088A000BA43826081F3108820202860002020666F
:1088B000EFF31081012080F31088206802689A434A
:1088C000026081F31088606FFEF729FA022060666B
:1088D000308B718B401A81B22046FFF7E3FEF8BD62
:1088E000318B728B891A89B2728B002AF7D00029DA
:1088F000F5D0EFF31082012686F310880668FF2773
:108900002137BE43066082F31088EFF31082012006
:1089100080F310882068866876087600866082F387
:1089200010882020286000E013E000202066A06668
:10893000EFF31082012080F31088206805689D43C2
:10894000056082F31088022060662046FFF7AAFEC9
:10895000F8BDC50208D55B0206D5012000051062EE
:108960002046FFF7A0FEF8BD020607D50A0605D58A
:10897000E16E0029F7D020468847F8BD4006FCD5B7
:108980004806FAD5204602F0C5FFF8BD0F080000E2
:108990002001000445B7000810B50446002C03D0A0
:1089A000E06F002802D007E0012010BD00217820F0
:1089B0000155204600F064F82420E0672068016833
:1089C000490849000160204603F0A6F8012819D0A3
:1089D000606A002802D0204602F0E6FD2068416867
:1089E0000922D20291434160206881682A22914382
:1089F000816020680168012211430160204602F075
:108A000039FE10BD012010BD10B502681748184985
:108A100082420BD1886B0122920490438863032128
:108A200089021448FEF7ACFA1D200EE0124B052017
:108A300000079A420CD14A6B01239B039A434A6375
:108A400003214902FEF79CFA1B20FEF7B1FD10BD81
:108A50000A4B9A42FBD18A6B01235B049A438A63D7
:108A60000C21FEF78DFA1C20EFE7000000480040C3
:108A70000010024000040050003801400044004053
:108A8000F0B587B0044614216846FCF790FB314AE4
:108A9000266800253048022103230424964218D179
:108AA000826B4E0432438263C26A0A43C262C06A66
:108AB0006A4608400590980223C218C269462748B2
:108AC000FEF7E8FA002211461D20FEF78DFD1D205D
:108AD0001CE0234F0122BE421CD1456B9603354357
:108AE0004563C56A1543C562C06A6D46104005906E
:108AF000032040021FC5052069460007FEF7CAFA99
:108B0000002211461B20FEF76FFD1B20FEF760FDC3
:108B100007B0F0BD134FBE42FAD1866B01277F0428
:108B20003E438663C66A1643C662C06A6E46C00785
:108B3000C00F05900C2023C6052018C66946000703
:108B4000FEF7A8FA002211461C20FEF74DFD1C205E
:108B5000DCE7000000480040001002400004005024
:108B6000003801400044004070B580231B58202B82
:108B700001D0022070BD00290AD0002A08D00124AB
:108B800083682403A34209D10369002B02D005E0C6
:108B9000012070BDCB0701D0012070BD002303660A
:108BA0000A4C0368A3420ED05C6824020BD5EFF395
:108BB0001084012585F310881D680126B60635430B
:108BC0001D6084F3108803F0E1F870BD0048004098
:108BD00070B580231B58202B01D0022070BD0029C6
:108BE0000AD0002A08D0012483682403A34209D1B3
:108BF0000369002B02D005E0012070BDCB0701D036
:108C0000012070BD002303660A4C0368A3420ED006
:108C10005C6824020BD5EFF31084012585F31088DE
:108C20001D680126B60635431D6084F3108803F0E5
:108C300005F970BD0048004010B503F065FB10BD9C
:108C40007047FFB583B004460F461546E06F2028F5
:108C500002D0022007B0F0BD002F0AD0002D08D0AE
:108C60000120A168000381420BD12069002803D0B4
:108C700007E0012007B0F0BDF80702D0012007B0DF
:108C8000F0BD0021842001512120E067FEF7CAFADF
:108C9000029026464036358275820120A168000385
:108CA000814202D12069002813D03D460027708AF6
:108CB00000281CD006980090002280212046029BAC
:108CC00003F08CF9002806D02020E067032007B0CD
:108CD000F0BD0025EBE7002D18D0216828788862C8
:108CE0006D1C708A401E7082708A0028E2D106983E
:108CF0000090002240212046029B03F06FF90028DB
:108D00000BD02020E067032007B0F0BD3888216831
:108D1000C005C00D8862BF1CE3E72020E06700208B
:108D200007B0F0BD70B50446E06F202801D00220E6
:108D300070BD00290AD0002A08D00123A0681B03B7
:108D4000984209D12069002802D005E0012070BDB9
:108D5000C80701D0012070BDE16420464030028286
:108D6000428200214030054641602120E067206FAB
:108D700000281AD0154BC362236F15481863236F60
:108D800014485863206F8163206813462830266F8B
:108D900002463046E16CFEF70CF8002805D01020A2
:108DA00068602020E067012070BD216840200862D3
:108DB000EFF31081012080F31088206882688023FF
:108DC0001A43826081F31088002070BD5FB80008EC
:108DD000ABB8000859B7000830B4C36F202B02D0DD
:108DE00030BC0220704700290AD0002A08D0012494
:108DF00083682403A3420BD10569002D03D007E04B
:108E000030BC01207047CD0702D030BC0120704734
:108E1000C164014640310A824A820021C16684222F
:108E200011502121C167A34202D10169002910D04C
:108E30000949C166EFF31081012282F310880068AE
:108E4000026880231A43026081F3108830BC00203E
:108E500070470249C166EDE77FBF00081DBF0008EB
:108E600010B503F0E9FA10BD704700000020014979
:108E700008707047B0030020012001490870704756
:108E8000B003002070B504460D46204600F02CF8D3
:108E9000012801D1801E70BD2268501CE168FCF7DA
:108EA00027F92160236921685943A368C818294616
:108EB0002269FCF763F90020EDE710B58160C2601C
:108EC0000361012444600024046010BD10B5044611
:108ED0002268501CE168FCF70BF96068814201D1FF
:108EE000012010BD0020FCE710B504462268901C4C
:108EF000E168FCF7FDF86068814201D1012010BDF6
:108F00000020FCE770B504460D462046FFF7DEFF63
:108F1000012801D1801E70BD236960685843A36891
:108F2000C11828462269FCF729F96268501CE168DB
:108F3000FCF7DEF861600020EDE770B504460D46F1
:108F4000002C01D1401E70BD00BF2068A842FCD398
:108F50002068401B206062685019E168FCF7C8F87F
:108F600061600020EFE770B504460D46002C01D18A
:108F7000401E70BD20684019206000BFE168206875
:108F80008842FBD8A2685019E168FCF7B1F8A160EB
:108F90000020EEE7FFB581B004460D4616460027D7
:108FA000002E06D00498002803D0E168206888428B
:108FB00003D30020C04305B0F0BD2168E068401A2B
:108FC000A84202D20020C043F5E7A0684019E1683A
:108FD00088420BD9A168E068471A2168E068401A06
:108FE000E919884202D20020C043E4E7A268D01900
:108FF000E168FCF77DF83160791904980160002080
:10900000D9E70146486870470146886870470246BC
:10901000002A01D1401E704700205060906010600F
:10902000D16000BFF7E70146002901D10120704758
:109030000868002801D10120F9E70020F7E7014680
:10904000002901D1012070470A68C868904201D107
:109050000120F8E70020F6E70FB400B50D48FFB097
:10906000007882B0012805D000207FB002B008BC93
:1090700004B01847012183AB49026846829A03F085
:10908000A5FA6846FCF7B2F802466946002003F0EC
:1090900067F9EAE78800002010B5064A1278012A2D
:1090A00001D0002010BD0A460146002003F058F907
:1090B00010BD0000880000200349096801600221FA
:1090C00081710149086070472001002000BFEFF363
:1090D0000580002800D0704707480068002804D1A8
:1090E000012080F3108800BF00BF03480068401CC7
:1090F0000149086000BFEEE70C01002070B504468E
:109100000D4600F04FF800280FD000F04BF80B216F
:10911000C90140180069002807D000F043F80B226D
:10912000D2018018016902A08847002070BD0000AC
:109130001B5B481B5B4A000070B502460C460021D1
:109140000023002A01D0002C02D10020C04370BDB2
:109150000021002316E0C8000D4D2858002810D12A
:10916000D8001058CD000A4E7051D80080184068C1
:10917000CD00AD19686007480068401C054D2860A7
:109180005B1C491C502901D2A342E4D30020DEE736
:109190002C010020280100200148006870470000D1
:1091A00028010020014800687047000024010020C9
:1091B000F8B506460F46002536E0002418E0FFF714
:1091C000F1FF002813D0FFF7EDFF0B21C901401874
:1091D000006900280BD0FFF7E5FF0B23DB01C01867
:1091E00002692819C000134B195813A09047641C3A
:1091F000052C04DAFFF7D0FF29198842DFD8FFF7E2
:10920000D1FF00280FD0FFF7CDFF0B21C901401877
:109210000069002807D0FFF7C5FF0B22D201801894
:10922000016907A088476D1DFFF7B6FFA842C4D8A3
:109230000020F8BD2C010020252D313673000000E0
:109240000D0A00000146202902D30020C0437047C8
:10925000012218204843044B1A500022182048438A
:10926000C01882600020F2E7A029002070B50546F2
:109270000024002D01D1401E70BD00240CE01820F8
:1092800060430C490858002805D10121182060438B
:10929000084A115002E0641C202CF0D300BF202C9F
:1092A00005D105A0FFF7D8FE0020C043E4E72C60FD
:1092B0000020E1E7A029002074696D65722049440F
:1092C0002069732066756C6C0D0A000010B50024CF
:1092D00000BF41E0182060432149085802283AD1D4
:1092E00018206043401880681E490968091A182030
:1092F00060431B4A8018C06881422CD91820604303
:10930000114640184069002820D0182060434018BA
:109310000079002804D101211820604311500AE08F
:109320000221182060430E4A11500E48016818208F
:1093300060438018816018226243094BD21810697B
:1093400018226243D2185169884704E0012118208D
:109350006043034A1150641C202CBBD310BD000095
:10936000A029002010010020F0B50446059D202C06
:1093700002D30020C043F0BD0226182060430E4FE8
:109380003E50182060433E46801901710B48066824
:1093900018206043C0198660182060433E4680193B
:1093A000C26018206043801943611820604380190F
:1093B00005610020DFE70000A02900201001002047
:1093C00007480068401C0649086006480268406873
:1093D0000021521C484103490A6048607047000060
:1093E000100100201801002000BFEFF305800028C5
:1093F00000D0704709480068002804D0074800687A
:10940000401E0649086005480068002804D100BFD6
:1094100080F3108800BF00BF00BFEAE70C01002006
:1094200070B504460D4629462046FBF7C0FE70BDC8
:109430000146302904DB392902DC084630380EE0C9
:10944000412904DB462902DC0846373807E0612958
:1094500004DB662902DC0846573800E00020C0B271
:10946000704710B502460B46002406E01078FFF75F
:10947000DFFF21014418521C5B1E002BF6D1204651
:1094800010BD0FB4F0B585B0044600200490002252
:109490002020039000200290002C02D00C9800287D
:1094A00005D1002005B0F0BC08BC04B018470DA8D9
:1094B0000490CFE0002908D10C980078252803D12A
:1094C0000C984078652800D0C9E00C9800782528D1
:1094D0006ED10C98401C0C900C98007803900C985E
:1094E000401C0C900398652877D004DC2A2807D00C
:1094F000642873D113E0702872D07828F9D13EE047
:1095000008E020780C9B1B78984202D0641C491E0E
:1095100000E001E00029F4D100BF521C88E00026E1
:1095200001960096002300252020049E20CE04965C
:1095300018E02078009E002E05D12D2803D10126A9
:10954000019600960CE0302809DB392807DC01265B
:1095500000960A265E430746303FF31900E003E019
:10956000641C491E0029E4D100BF019E012E01D1D7
:10957000DE43731C002D00D02B60521C58E00023EA
:109580000025049E20CE04961FE02078302806DBBC
:10959000392804DC1E010746303FF31913E0612827
:1095A00007DB662805DC1F010646573EBB190AE0AB
:1095B00043E0412806DB462804DC1F010646373E0F
:1095C000BB1900E003E0641C491E0029DDD100BF87
:1095D000002D00D02B60521C2AE01BE024E0FFE7A6
:1095E000049E01CE049600250023254609E0267836
:1095F0000C9F3F78BE4201D05B1C00E003E0641C7E
:10960000491E0029F3D100BF002801D00560436046
:10961000521C0DE0049B01CB0493002800D0046091
:10962000521C0123029303E001200290002200BF9C
:1096300000BF029801280DD111E020780C9B1B7807
:10964000984205D1641C0C98401C0C90491E01E006
:10965000002204E00C980078002800D02AE700BF20
:109660000020049010461DE70FB4F8B506460C46DE
:10967000002509A8009021463046009B089A02F078
:10968000A5FF054600200090A54200D3651E284690
:10969000F8BC08BC04B01847FEB504460F46154692
:1096A0000026002001900090002C01D0002D01D157
:1096B0000020FEBD2846FBF799FD009000988742E8
:1096C00001D20020F5E70098381A0190002609E041
:1096D000A0192946009AFBF790FD002801D1A01996
:1096E000E7E7761C01988642F2D30020E1E770B5E7
:1096F00004460D46002C01D0002D02D10020C043AD
:1097000070BD012120461030FFF717FC20462030A5
:10971000A968FFF712FC0020F2E770B504460D4679
:10972000002C01D0002D02D10020C04370BD0121CA
:1097300020461030FFF717FC20462030A968FFF7BD
:1097400012FC0020F2E710B50446002C00D110BD39
:1097500020461030FFF767FC012801D10020F6E712
:1097600020462030FFF75FFC012801D10020EEE702
:1097700020461030FFF745FC0C2148432168401873
:10978000E5E77CB504460E460025002001900090D8
:10979000002C00D17CBD20461030FFF750FC002883
:1097A00001D00020F6E76B4601AA31462046203062
:1097B000FFF7F0FB002801D00020EBE72046103037
:1097C000FFF722FC0C21484321684518A068019945
:1097D000401828606E600098A8602846DAE7FFB558
:1097E00081B004460E461D4600270C2068430399AD
:1097F000884202D3781E05B0F0BD0C202F464743A7
:109800002660676060688019A0600398C11BE160F2
:10981000294620461030FFF7FAFB20462030E16849
:10982000FFF7F5FB0020E6E7FEE7000010B50E4C61
:10983000002208212046FDF7EEFC002210212046E0
:10984000FDF7E9FC0A2003F09FFB012208212046D6
:10985000FDF7E1FC0A2003F097FB002208212046D7
:10986000FDF7D9FC10BD00000004005010B50E4CEF
:10987000002208212046FDF7CEFC012210212046BF
:10988000FDF7C9FC0A2003F07FFB012208212046D6
:10989000FDF7C1FC0A2003F077FB002208212046D7
:1098A000FDF7B9FC10BD000000040050F8B500241D
:1098B000144E07462546002208213046FDF7ABFC32
:1098C0000A2003F061FB012208213046FDF7A3FCCA
:1098D0006006040E10213046FDF796FC002801D0EA
:1098E000641CE4B2052003F04FFB6D1CEDB2082DA3
:1098F000E1D3002F03D0FFF799FF2046F8BDFFF713
:10990000B5FFFAE70004005070B5154E0546002279
:1099100008213046FDF77FFC0024E80901D0012230
:1099200000E0002210213046FDF775FC6806050EA8
:109930000A2003F029FB012208213046FDF76BFCC9
:109940000A2003F021FB002208213046FDF763FCCA
:109950000A2003F019FB641CE4B2082CDDD370BDAF
:109960000004005010B50C4C012210212046FDF7D8
:1099700052FC012208212046FDF74DFC0022102157
:109980002046FDF748FC0A2003F0FEFA00220821D9
:109990002046FDF740FC10BD0004005010B50E4CF1
:1099A000002208212046FDF736FC00221021204627
:1099B000FDF731FC0A2003F0E7FA012208212046D6
:1099C000FDF729FC012210212046FDF724FC0A2086
:1099D00003F0DAFA10BD00000004005070B5144D19
:1099E0000024012210212846FDF715FC062003F073
:1099F000CBFA012208212846FDF70DFC062003F0D2
:109A0000C3FA07E0641CE4B2FA2C03D9FFF7C6FFDF
:109A1000012070BD10212846FDF7F6FB0028F1D18A
:109A2000002208212846FDF7F6FB002070BD00004B
:109A30000004005010B5FCF765FC10BD70B500F0D7
:109A40002FF80025104C012818D1A078002815D136
:109A50000120A0700D480E49056020780D4B0E4A7C
:109A60000E4E5A2802D3FF20000401E0FF2000021E
:109A700008601B681268316801F058F900F010F8AE
:109A8000002800D1A57070BD380000202C000020F7
:109A900024000020180000201C00002020000020CE
:109AA00010B5044881880068FDF7AEFB012800D09E
:109AB000002010BD5400002010B53721202000F0F8
:109AC00070F80321212000F06CF84021222000F0E2
:109AD00068F80821232000F064F8AA21302000F063
:109AE00060F80A4802210187322000F05AF801216B
:109AF000332000F056F85F21202000F052F804488F
:109B000000F008F80A2003F03FFA10BD74060020A8
:109B1000DB00002010B501460F2000F021F80028DE
:109B200000D0012010BD10B50446FFF71BFF322006
:109B3000FFF7EAFEFFF752FFE0B2FFF7E5FEFFF79F
:109B40004DFFFFF70FFF3320FFF7DEFEFFF746FF65
:109B50000020FFF7ABFE0446FFF720FF204610BDB4
:109B600010B50C46FFF7DFFF2070012010BD70B567
:109B70000D460446FFF7F6FE3220FFF7C5FEFFF75D
:109B80002DFFE0B2FFF7C0FEFFF728FF2846FFF7E2
:109B9000BBFEFFF723FFFFF701FF0A2003F0F4F9F4
:109BA00070BD10B5FFF7E3FF012010BD10B50248EE
:109BB000FDF7CCFB10BD000014040020F0B583B00D
:109BC00004460026EFF310800090012080F31088F7
:109BD000344B2068C21804D13349CE68032189046C
:109BE0000E4081680291C168019141698569002A2E
:109BF00007D12E48826AC7043A438262826ABA4316
:109C00008262084628433CD026482268C24205D1D9
:109C10002548C368032292049343C3602746203734
:109C2000002910D02068026901231A4302612068CC
:109C300041610821204600F03BF8032800D1B873A9
:109C4000216808204860002D10D020680169012299
:109C500011430161206885611021204600F028F839
:109C6000032800D1B8732168102048600D4821688E
:109C7000C14206D10C48C16803229204914331438A
:109C8000C1602068016949084900016121680298A2
:109C9000886021680198C860009880F3108803B03C
:109CA000F0BD00000084FFBF4010024000100240E1
:109CB00070B506460D4600240B480A490068FBF7BC
:109CC00017FA7D21C90048433268401E002800D1A0
:109CD000032413682946994301D00028F5D1204672
:109CE00070BD0000204E00000801002010B50248A1
:109CF000FEF700FD10BD00004404002010B5032055
:109D000000F002F810BD000070B5164D00262C467C
:109D1000103C002811D021468978032814D001284E
:109D20000AD1491CC8B2A0700C2817D204280FD041
:109D30008000285800F0B0F970BD00F05DFA0520F1
:109D4000FDF770F8A67001E00029F5D12868F1E769
:109D500005492869096800F09FF970BD00F042FAD2
:109D600070BD0000A40000206000002000B587B096
:109D7000012069464870022008700E490191410295
:109D800002910D49039180210491059069460120BB
:109D900002F0CEF90948FFF769FA00F02DFA00F059
:109DA0006BF96420FDF73EF80020FFF7ADFF0020BF
:109DB00007B000BD2C2300202C2700209C00002091
:109DC000034880780C2801D000207047012070479C
:109DD00094000020032802D30020C0437047C30032
:109DE0000248C150181882800020704714230020B8
:109DF000FEB5002568460571058105805D4F5E4C06
:109E00005E4EA0E06846007900F0EAF86846017905
:109E100030782154401C307020785528F1D160787A
:109E2000AA28EED1607A5528EBD1A07AAA28E8D1E9
:109E30006068029052496846008909688842E0D10A
:109E4000A079012814D1E07901287CD1207A00285A
:109E500079D14C4805604C4805704C4805704CA0C1
:109E6000FFF7FAF8FF2101314348FBF7A0F93570FD
:109E7000A079022806D0032818D0052826D0042867
:109E800061D141E03C496846CA790270097A417063
:109E900000883C2802D83C2069460880684604882F
:109EA000BC8403F03FFA21463DA026E032496846D3
:109EB000CA790270097A417000880A2802D80A20FB
:109EC00069460880684604887C8712E02A4968460B
:109ED000CA790270097A417001887D20C000081A91
:109EE0003649884202D33648694608806846048865
:109EF000FC8003F017FA214632A0FFF7ADF864208A
:109F000003F03BF802F0B6FB1B486946C2790A70C1
:109F1000007A487008880A2801D80A2002E06428DC
:109F200001D96420088008883071012070711648BA
:109F3000FF210570154801310570124805600E4873
:109F4000FBF735F9357001A9012002F0B1F80028BE
:109F500000D157E7FFF734FF012809D1F078002836
:109F600006D0FF2101310448FBF721F9F570357067
:109F7000FEBD000074060020142200209400002082
:109F8000600000205C0000203B0000203C0000201E
:109F9000CAD5B5BD475053B5C44F4B0D0A0000009C
:109FA000CAD5B5BDD0DEB8C4475053BFAAB9D8CAC8
:109FB000B1BCE43A25640D0A00000000292300002A
:109FC00010270000CAD5B5BDD0DEB8C4BEB2D6B920
:109FD000D0DDC3DFCAB1BCE43A25640D0A0000003D
:109FE00070B51E491E4B4A78012A05D1CA687F2ADE
:109FF00002D29854521CCA6000220A2802D00D28AE
:10A0000004D029E00120CA60487025E04A70CC687D
:10A01000002C21D018192038C277114D8868FFF71D
:10A0200011F910A221462846FFF736FB002805D07B
:10A0300029460DA0FFF710F801200BE00CA22146E5
:10A040002846FFF729FB002806D0294606A0FFF77F
:10A0500003F80220FFF758FE002070BD9400002096
:10A06000AC2700206F6B00005B525D2025730A0057
:10A070006572726F7200000010B50348012281887A
:10A080000068FDF7C8F810BD1423002010B50020AB
:10A09000FFF73AFE10BD00000FB430B591B015AB1C
:10A0A000402101A8149A02F091FA002501A8FBF7BB
:10A0B0009DF8024601A9012002F052F904460A481F
:10A0C0007D220095074B120100218068FFF74CF9B3
:10A0D00001A906A0FEF7C0FF204611B030BC08BCA5
:10A0E00004B01847FD9C0008940000205B535D20DD
:10A0F00025730A0070B505460C480C4680780C287C
:10A1000002D00020C04370BD00F076F80520FCF7B7
:10A1100089FE22462946012002F022F90520FCF79B
:10A1200081FE00F05FF8002070BD00009400002068
:10A13000F8B51F4E1F4C30682169401A0A2836D9DD
:10A14000E078002833D0012020711B4801781B489B
:10A15000FFF7D0FFFF2101311948FBF728F8194814
:10A160000025057030682061E079FF21401CE07116
:10A170001548174E01601548164F03683268386855
:10A1800000F0D4FD6420FCF74DFE0F482946056021
:10A190000E4832680368386800F0C8FDE07904288A
:10A1A00002D92571E570E5710BA0FEF755FFF8BDEA
:10A1B00028000020380000208E000020EC11002034
:10A1C000142200209400002020000020180000200D
:10A1D0001C000020240000206C6F726120627566F4
:10A1E000610D0A0010B50348002281898068FDF7DF
:10A1F00012F810BD1423002010B5034801228189F4
:10A200008068FDF708F810BD142300201CB500215C
:10A2100018480091164A01910260C163120542601C
:10A22000816007228263012202610246C1602032FE
:10A230001170FF235170C233436281621173016355
:10A240008161042241634261C161FCF78FFB0028F8
:10A2500001D072B6FEE7084800908013019069466D
:10A260000448FCF7D5FA002801D072B6FEE71CBD01
:10A2700000240140B803002002000004F0B587B0BC
:10A2800014216846FAF793FF4148C26A04210A4341
:10A29000C262C26A0A400592C16A01252943C162AD
:10A2A000C16A29400591C26A02210A43C262C06A9A
:10A2B000052708403F070590002236493846FCF73D
:10A2C000AAFF002234493548FCF7A5FF01221103FB
:10A2D0003846FCF7A0FF012240213048FCF79BFFE5
:10A2E00011263604002469463846019600950294EA
:10A2F000FCF7D0FE2A480090029469460195039429
:10A300003846FCF7C7FE2448029418380090694686
:10A31000019503942148FCF7BDFEA22000906946F8
:10A32000019602941D48FCF7B5FE09200003009039
:10A330000194694602941948FCF7ACFE182000907D
:10A34000112001900294694603941448FCF7A2FE80
:10A3500040200090032003900195029469460F4825
:10A36000FCF798FE2802FCF763FF00221146052047
:10A37000FDF73AF90520FDF72BF9002211460720D9
:10A38000FDF732F90720FDF723F907B0F0BD000013
:10A3900000100240108900001D4100000004005020
:10A3A0001099000010B5FFF731FF00F009F800F038
:10A3B00099F800F0B3F800F01FF800F043F810BD72
:10A3C00010B50C480A490160E121490241600021B1
:10A3D0008160C160016181610C2201624261416260
:10A3E000FEF7DAFA002801D072B6FEE710BD0000D1
:10A3F000004800404404002010B5114C0F48206074
:10A40000FF20053060600020A060E0602061606196
:10A41000E0610121206249026062A161A06207201F
:10A42000E0622046FDF70FFE002801D072B6FEE77D
:10A430002068016840221143016010BD00300140D6
:10A44000DC05002010B58AB000240494059406941D
:10A4500007940894224809940094019402941F4997
:10A46000039401601F21846041600461F92144610B
:10A47000C160FDF7F9FE002801D072B6FEE70120A9
:10A480000003049004A91648FDF770FF002801D0CE
:10A4900072B6FEE71248FEF775F8002801D072B6D2
:10A4A000FEE7089408A90E480994FDF78FFE0028DE
:10A4B00001D072B6FEE76020009001940294002261
:10A4C000694603940648FDF7EDFF002801D072B6F7
:10A4D000FEE70348FDF7BEFF0AB010BD00080140CB
:10A4E0003406002010B50C480A490160E1214902F8
:10A4F000416000218160C16001618161C1610C2204
:10A50000016242614162FEF747FA002801D072B64B
:10A51000FEE710BD00380140CC04002010B50C4807
:10A520000A4901604B21C901416000218160C1607D
:10A5300001618161C1610C22016242614162FEF7E9
:10A540002BFA002801D072B6FEE710BD004400408F
:10A5500054050020FEE7704710B5044800228189A9
:10A560008068FCF758FEFCF705F910BD04220020B6
:10A5700010B50448012281898068FCF74CFEFCF785
:10A58000FFF810BD04220020C3000248C150181873
:10A590008280704704220020F0B585B04848FCF75F
:10A5A00085F94848FDF738FD4748FDF741FE474823
:10A5B000FEF77AF84648FEF777F84648FEF774F853
:10A5C00000F0D0FB14216846FAF7F1FD00241026B4
:10A5D000112705200294694600070197009603940D
:10A5E000FCF758FDF5010520029469460007019724
:10A5F00000950394FCF74EFDFDF7E0FD3648816BB6
:10A60000020411438163354801680422114301604B
:10A6100001210846FDF712F8FDF7F6FC00F064FE94
:10A62000FFF7C0FE002001F0FDFD012001F0FAFD62
:10A63000022001F0F7FD00960126052002946946EC
:10A64000000701960394FCF725FD05200122102147
:10A650000007FCF7E0FD052002946946000701961B
:10A6600000950394FCF716FD0520012229460007FA
:10A67000FCF7D1FD1A48007800281CD1194C20683D
:10A68000C10718D1184D2968884214D0174801789D
:10A690001748142901D3FF2101E0FF2109020160BD
:10A6A000144900680B6814490A681449096800F0E5
:10A6B0003DFB2068286012A0FEF7CEFC05B0F0BD7F
:10A6C000B8030020DC0500203406002044040020EC
:10A6D000CC0400205405002000100240007000400F
:10A6E0003000002028000020340000203800002026
:10A6F00024000020180000201C0000202000002062
:10A7000077616B752075700D0A000000F8B502F0D6
:10A71000C5FD754800F0CAFA744CE0807248801C90
:10A7200000F0C4FA20817048001D00F0BFFA60817B
:10A7300070486F494180818C002902D1E1210901D3
:10A740008184418F6C4A002901D0914201D96B4923
:10A7500041878BB2818C8B4202D2FF312D314187F0
:10A76000C3887D21C900591A654B994200D3C28024
:10A77000604D60484035297961700091614AC18E11
:10A780001170614AC18F1170604A818F1170A9796F
:10A7900021705F4A817A11705E4986880E605E4A38
:10A7A00005211180C7883846FAF7A2FC5B4908806A
:10A7B00001463046FAF79CFC8800081886B25848D3
:10A7C00006807D20C0007043FAF7A4FF554A564B1F
:10A7D000FAF728FFFAF7C0FF54490880544806806A
:10A7E00054480188C820FAF783FC534900260880A2
:10A7F000524901200880A7800099002906D17D21B7
:10A80000C900A18040490870404806707D20A18899
:10A81000C000FAF76DFC47490022088048494948C2
:10A82000FCF76AFE002801D072B6FEE7A88C01286A
:10A8300005D0688C444C454F012838D03FE0FF20BC
:10A84000000203461A46114600F070FAFF24F53460
:10A850002046FCF7E7FAFF20000403461A4611469B
:10A8600000F064FA2046FCF7DDFA00231A46194688
:10A87000184600F05BFA2046FCF7D4FA34486946E3
:10A88000088072B68021334C2046FBF76FFD00280C
:10A8900004D0022269462046FBF70EFE62B6AE8463
:10A8A00002F040FD642002F068FB01F0D5FE00F0EC
:10A8B000CBF902F037FD642002F05FFBFC60288CCE
:10A8C000012806D12E8402F02DFD642002F055FBF4
:10A8D000FC600848204A0188914202D1C0880028C3
:10A8E00000D1FC60F8BD0000004F0008000000200F
:10A8F0000902000074060020102700003C0F000031
:10A9000029230000F00000207200002073000020C6
:10A910006400002060000020680000206A00002021
:10A9200066000020F853E3A59B843E406C000020A5
:10A93000700000206E0000207600002074000020CF
:10A94000FF7F0000140400200400FA0500ED00E081
:10A95000AAAA0000384A0008AA55000000B5044918
:10A9600040208862FF20F53002F0F8FC00BD0000B6
:10A9700000040050FF2302461B0200B519020D48D7
:10A980009A4202D100F0C0F800BD8A4202D100F024
:10A9900057F809E0FF2A04D0824205D100F002F9FD
:10A9A00000BD00F009F800BD002AFCD100F07AF8E3
:10A9B00000BD0000FFFFFF0000B500F02FF800F021
:10A9C0002DF800F02BF800F029F800F027F800F03F
:10A9D00025F800F023F800F021F800F01FF800F04F
:10A9E0001DF800F01BF800F019F800F017F800F05F
:10A9F00015F800F013F800F011F800F0B7F800F0C7
:10AA0000B5F800F0B3F800F0B1F800F0AFF800F0DE
:10AA1000ADF800F0ABF800F0A9F800BD0748402100
:10AA2000816100BF00BF00BF00BF00BF00BF8162E7
:10AA300000BF00BF00BF00BF00BF70470004005050
:10AA400000B500F093F800F091F800F08FF800F0F6
:10AA50008DF800F08BF800F089F800F087F800F02E
:10AA600085F8FFF7DBFFFFF7D9FFFFF7D7FFFFF709
:10AA7000D5FFFFF7D3FFFFF7D1FFFFF7CFFFFFF7BA
:10AA8000CDFFFFF7CBFFFFF7C9FFFFF7C7FFFFF7CA
:10AA9000C5FFFFF7C3FFFFF7C1FFFFF7BFFFFFF7DA
:10AAA000BDFF00BD00B5FFF7B9FFFFF7B7FFFFF728
:10AAB000B5FFFFF7B3FFFFF7B1FFFFF7AFFFFFF7FA
:10AAC000ADFFFFF7ABFFFFF7A9FFFFF7A7FFFFF70A
:10AAD000A5FFFFF7A3FFFFF7A1FFFFF79FFFFFF71A
:10AAE0009DFFFFF79BFFFFF799FFFFF797FFFFF72A
:10AAF00095FFFFF793FFFFF791FFFFF78FFFFFF73A
:10AB00008DFFFFF78BFF00BD00B5FFF787FFFFF755
:10AB100085FFFFF783FFFFF781FFFFF77FFFFFF759
:10AB20007DFFFFF77BFFFFF779FF00F01FF800F0D4
:10AB30001DF800F01BF800F019F800F017F800F00D
:10AB400015F800F013F800F011F8FFF767FFFFF7B2
:10AB500065FFFFF763FFFFF761FFFFF75FFFFFF799
:10AB60005DFFFFF75BFFFFF759FF00BD0C48402179
:10AB7000816100BF00BF00BF00BF00BF00BF00BFBA
:10AB800000BF00BF00BF00BF00BF00BF00BF00BFCD
:10AB9000816200BF00BF00BF00BF00BF7047000060
:10ABA0000004005000B5FFF7E1FFFFF7DFFFFFF7FC
:10ABB000DDFFFFF7DBFFFFF7D9FFFFF7D7FFFFF759
:10ABC000D5FFFFF7D3FFFFF7D1FFFFF7CFFFFFF769
:10ABD000CDFFFFF7CBFFFFF7C9FFFFF7C7FFFFF779
:10ABE000C5FFFFF7C3FFFFF7C1FFFFF7BFFFFFF789
:10ABF000BDFFFFF7BBFFFFF7B9FFFFF7B7FFFFF799
:10AC0000B5FFFFF7B3FF00BD08B5002808D0024626
:10AC1000002106480091044B0068FEF7A5FB08BD23
:10AC2000002000F005F808BD31AC0008D400002079
:10AC3000044972B60248C860BFF34F8F70470000E6
:10AC40000400FA0500ED00E010B514481249018037
:10AC5000134981801349C1800A2303810021418166
:10AC600081810122C28181834324C4860224048716
:10AC70000D4C44878287C28702464032118451843A
:10AC80009184C1839180142484821182E12109017D
:10AC90008184038410BD0000AA55000074060020C2
:10ACA00034120000102700003C0F0000008870479D
:10ACB00070470000F8B5044600206A461080194D20
:10ACC00055222A70AA226A700322AA70661DEE70AD
:10ACD0002A716971144A49008918AC712246E81D2D
:10ACE000FAF74CFA002007E029186A46897812889A
:10ACF00089186A461180401CB042F5DB611DA81C12
:10AD0000FBF77CFA01466846018029190078C87172
:10AD1000684640780872224609320249002001F054
:10AD20001FFBF8BDD80A002074060020F8B51646AF
:10AD300004460F46012205201D46D1030007FCF7FB
:10AD40006AFAFFF70BFE3846FFF714FE3046FFF7AE
:10AD500011FE2846FFF70EFE2046FFF70BFEFFF719
:10AD6000FDFDF8BD10B5012105200022C903000733
:10AD7000FCF751FA10BD000010B5FBF7F9F9FEF72A
:10AD800011FA00280DD0FEF70DFA0B24E40100198A
:10AD90000069002805D0FEF705FA0019016902A034
:10ADA0008847002010BD00004F4B0D0A0000000036
:10ADB00010B5FBF7FBF9FEF7F5F900280DD0FEF70B
:10ADC000F1F90B24E40100190069002805D0FEF711
:10ADD000E9F90019016902A08847002010BD0000B0
:10ADE0004F4B0D0A0000000010B5022814DAFEF7E0
:10ADF000D9F900280DD0FEF7D5F90B24E40100198C
:10AE00000069002805D0FEF7CDF90019016907A0F7
:10AE100088470020C04310BD4868FAF7FBF90028B6
:10AE200001D1FEF723F8002010BD000064656275B3
:10AE3000675F6F666620666C61670D0A0000000040
:10AE400010B5022814DAFEF7ADF900280DD0FEF790
:10AE5000A9F90B24E40100190069002805D0FEF7C8
:10AE6000A1F90019016907A088470020C04310BD5F
:10AE70004868FAF7CFF9002801D1FDF7FDFF00205F
:10AE800010BD000064656275675F6F6E20666C615F
:10AE9000670D0A0010B5FFF75FFBFEF783F9002886
:10AEA0000DD0FEF77FF90B24E4010019006900289A
:10AEB00005D0FEF777F90019016902A08847002044
:10AEC00010BD00004F4B0D0A0000000010B5FFF749
:10AED0004FFBFEF767F900280DD0FEF763F90B244E
:10AEE000E40100190069002805D0FEF75BF900199C
:10AEF000016902A08847002010BD00004F4B0D0AD9
:10AF00000000000070B5FEF74DF90B25ED0100289B
:10AF10000CD0FEF747F940190069002806D0FEF76B
:10AF200041F9401902690FA111A09047FEF73AF9C3
:10AF3000002815D0FEF736F94019006900280FD017
:10AF4000FBF7ACF8FAF726FC04460E46FEF72AF9A2
:10AF5000401905690B482246017833460AA0A847E4
:10AF6000002070BD76312E302E302E3400000000CF
:10AF700056657273696F6E3A202020202020257359
:10AF80000D0A000038000020426174746572793A3D
:10AF90002020202020202575252520252E326656AC
:10AFA0000D0A000010B511210248FEF7C5F8002077
:10AFB00010BD000068D300080020704710B50728B6
:10AFC00014D0FEF7EFF800280DD0FEF7EBF80B24B5
:10AFD000E40100190069002805D0FEF7E3F8001924
:10AFE000016903A088470020C04310BD002010BDA8
:10AFF00075736167653A207274635F736574207955
:10B00000797979206D6D206464206868206D6D20E9
:10B0100073730D0A0000000010B50020FFF7F4FD67
:10B02000002010BD10B50B24E401062812DAFEF74B
:10B03000B9F800280BD0FEF7B5F800190069002810
:10B0400005D0FEF7AFF8001901690BA08847002072
:10B05000C04310BDFEF7A6F800280BD0FEF7A2F8FB
:10B0600000190069002805D0FEF79CF80019016955
:10B0700011A08847002010BD7365745F6164632070
:10B080006E6F726D616C5F6D696E206E6F726D6157
:10B090006C5F6D6178206572726F725F6D696E2092
:10B0A0006572726F725F6D6178206572726F725F28
:10B0B000636E740D0A0000004F4B0D0A0000000083
:10B0C00010B50B24E40102280FDAFEF76BF8002814
:10B0D0001BD0FEF767F800190069002815D0FEF7AD
:10B0E00061F8001901690AA00EE0FEF75BF800287C
:10B0F0000BD0FEF757F800190069002805D0FEF7BD
:10B1000051F80019016904A08847002010BD000013
:10B110004552524F520D0A004F4B0D0A00000000DD
:10B1200070B500250B24ED43E40102280FDAFEF789
:10B1300039F8002822D0FEF735F8001900690028F8
:10B140001CD0FEF72FF80019016916A015E0486819
:10B15000FAF760F8002801D0082811D9FEF722F884
:10B1600000280BD0FEF71EF800190069002805D052
:10B17000FEF718F8001901690EA08847284670BD2F
:10B18000FEF710F800280BD0FEF70CF80019006944
:10B19000002805D0FEF706F80019016908A08847C5
:10B1A000002070BD7365745F6465765F69642069B3
:10B1B000640D0A006964206572726F720D0A0000E6
:10B1C0004F4B0D0A0000000010B50B24E4010328CA
:10B1D00012DAFDF7E7FF00280BD0FDF7E3FF0019B7
:10B1E0000069002805D0FDF7DDFF001901690BA0FB
:10B1F00088470020C04310BDFDF7D4FF00280BD0C6
:10B20000FDF7D0FF00190069002805D0FDF7CAFF3F
:10B21000001901690AA08847002010BD7365745F9A
:10B220006970205B7365727665725F69705D205B23
:10B230007365727665725F706F72745D0D0A0000DF
:10B240004F4B0D0A0000000010B50B24E401032849
:10B2500012DAFDF7A7FF00280BD0FDF7A3FF0019B6
:10B260000069002805D0FDF79DFF001901690BA0BA
:10B2700088470020C04310BDFDF794FF00280BD085
:10B28000FDF790FF00190069002805D0FDF78AFF3F
:10B29000001901690AA08847002010BD7365745F1A
:10B2A00077696669205B737369645D205B706173A5
:10B2B00073776F72645D205B69705D0D0A0000003A
:10B2C0004F4B0D0A0000000010B5FFF765F9002094
:10B2D00010BD10B5FEF7DAFE002010BD10B5FEF768
:10B2E0006FF8FBF7B3FF10BD10B59AB03421684674
:10B2F000F9F75DFF142115A8F9F759FF20210DA8D2
:10B30000F9F755FF234801680324E402A143C2145E
:10B3100089180160FCF78AF91F480169214301611E
:10B320000E200090FF200130029010200490022097
:10B330000990400401210B900001059100240C901C
:10B3400003910A946846FCF7E5FB002801D072B629
:10B35000FEE70F20159003201690179418940121F2
:10B36000199415A8FCF768FA002801D072B6FEE718
:10B3700087200D9003200F94800414901094119452
:10B380000DA8FCF78FF9002801D072B6FEE71AB0BD
:10B3900010BD00000070004040100240024901480A
:10B3A000886070470050000800ED00E0F0B40268CB
:10B3B0000124A407144D154E154FA04205D0A842F4
:10B3C00003D0B04201D0B84203D170239A434B68F6
:10B3D0001A43A04205D0A84203D0B04201D0B842DF
:10B3E00004D103231B029A43CB681A4380239A4358
:10B3F0000B691A4302608A68C2620968816201218E
:10B400004161F0BC704700000004004000080140AA
:10B410000014014010B4C906C90E01238B40046A10
:10B420009C430462036A8A401343036210BC704762
:10B4300030B48468FF252D02AC431B0213430B4339
:10B440002343836030BC7047826870239A430A4369
:10B4500007210A438260704730B4026A52085200E2
:10B460000262026A446883697025AB439B089B00B3
:10B470000D681D4302239A438B6813434460856122
:10B4800049684163036230BC704730B4026A1023DC
:10B490009A430262036A4568826907242403A2432F
:10B4A00003242402A2430C68240214432022934361
:10B4B0008A6812011A4345608461496881630262A7
:10B4C00030BC704730B4026AFF2301339A430262F2
:10B4D000026A4468C3697025AB439D08AD000B68E0
:10B4E0002B4301256D02AA438D682D02154344604C
:10B4F000C3614968C163056230BC704730B4026AF9
:10B5000001231B039A430262036A4568C269072448
:10B510002403A24303242402A2430C6824021443FC
:10B520000122520393438A6812031A434560C4619F
:10B5300049680164026230BC704730B4036A046A2F
:10B540006408640004628469F025AC43120122435C
:10B550000A24A3430B438261036230BC704730B4BA
:10B56000036A1024A34303628369046A0F252D0331
:10B57000AB4312031A43A0239C4309012143826178
:10B58000016230BC7047000010B505480549806A6B
:10B59000884204D3642001F0F0FC01F05DF810BD96
:10B5A00000000020002F0D0010B4818CC90707D0C7
:10B5B00001684A6801235B049A43836A1A434A601C
:10B5C000818C890707D501684A6801231B049A43C7
:10B5D000C36A1A434A60818C490707D501684A68E3
:10B5E00001239B049A43036B1A434A60818C090729
:10B5F00007D501684A680123DB039A43436B1A436A
:10B600004A60818CC90607D501688A6801231B033B
:10B610009A43836B1A438A60818C890607D5016837
:10B620008A6801235B039A43C36B1A438A60818C47
:10B63000490612D501684B6801221205046C934338
:10B6400023434B60016C914207D101684A68032390
:10B650005B059A43436C1A434A60818C090607D5FF
:10B6600001684A680123DB04806C9A4302434A6004
:10B6700010BC7047F0B583B00446264600278036DC
:10B680007760FBF7CFFD0290206800682546000731
:10B69000603500281CDA2A48009001210022490563
:10B6A0002046029B00F09AFC002811D0EFF3108195
:10B6B000012080F310882068026880239A4302608A
:10B6C00081F310882020E0672F76032003B0F0BDBF
:10B6D00020680068400729D5194800900121002200
:10B6E00089052046029B00F079FC00281ED0EFF36C
:10B6F0001081012080F3108820680268FF23213325
:10B700009A43026081F31088EFF31081012080F3E7
:10B7100010882068826852085200826081F3108885
:10B72000202030602F76032003B0F0BD2020E0679A
:10B730003060276667662F76002003B0F0BD0000FA
:10B74000FFFFFF0110B5806A0022014640314A83A5
:10B750004A82FCF7CBFF10BDF8B5846AE06F25463E
:10B7600080352E682168896800270906002906DAD5
:10B77000212804D152200753204600F0DFF820682A
:10B780008068400606D5222E04D15A200753204651
:10B7900000F090F868681021084368602046FCF7C4
:10B7A000A5FFF8BD70B50146886A096809680023DD
:10B7B0008906002937DB5A210B52EFF31082012151
:10B7C00081F3108801680C68FF250135AC430C60DB
:10B7D00082F31088EFF31082012181F31088016851
:10B7E0008C68640864008C6082F31088EFF3108228
:10B7F000012181F3108801688C684025AC438C607E
:10B8000082F31088202280210A50016E01290AD17A
:10B81000EFF3108281F3108801680C681025AC43A7
:10B820000C6082F310884366016E012902D0FDF797
:10B8300003FA70BD5821095AFCF734FF70BD10B5EA
:10B84000806A01214166016E012902D0FDF7F8F9F5
:10B8500010BD5821095A4908FCF724FF10BD10B546
:10B860000146886A0968096889061BD400225221AA
:10B870000A52EFF31082012181F3108801688B686E
:10B880008024A3438B6082F31088EFF310810122A0
:10B8900082F310880068026840231A43026081F333
:10B8A000108810BDFDF7DCFA10BD10B5806AFDF7F9
:10B8B000DBFA10BD10B4EFF31082012181F3108880
:10B8C00001680B68FF242134A3430B6082F31088C6
:10B8D000EFF31082012181F3108801688B685B0807
:10B8E0005B008B6082F31088016E01290AD1EFF3AF
:10B8F000108281F3108801680B681024A3430B6049
:10B9000082F31088202280210A500021016681667E
:10B9100010BC704710B5EFF31082012181F310883D
:10B9200001680B684024A3430B6082F31088202138
:10B93000C1670021C166FDF793FA10BD10B4EFF3A3
:10B940001082012181F3108801680B68C024A34391
:10B950000B6082F310882021C16710BC7047000083
:10B9600070B5014640318B8B024680321568144613
:10B970000268222D04D0906908210843906170BDAF
:10B98000526A456D1A402A80426D921C42654A8B6C
:10B99000521E4A834A8B002AF1D1EFF31083012211
:10B9A00082F3108802681568FF262136B5431560BA
:10B9B00083F31088EFF31083012282F3108802686A
:10B9C00095686D086D00956083F3108820222260D1
:10B9D000002484664466184B02689A420ED053686D
:10B9E0001B020BD5EFF31083012585F31088156832
:10B9F0000126B606B543156083F31088026E012A4E
:10BA000002D0FDF719F970BD0466EFF3108301222F
:10BA100082F31088026815681024A543156083F32B
:10BA200010880268D369DB43DB0600D41462098BFB
:10BA3000FCF738FE70BD00000048004070B50146BC
:10BA400040318B8B02468032156814460268222DE5
:10BA500004D0906908210843906170BD526A1A4071
:10BA6000436D1A70426D521C42654A8B521E4A83C6
:10BA70004A8B002AF1D1EFF31083012282F3108860
:10BA800002681568FF262136B543156083F31088D8
:10BA9000EFF31083012282F31088026895686D0825
:10BAA0006D00956083F31088202222600024846654
:10BAB0004466184B02689A420ED053681B020BD59D
:10BAC000EFF31083012585F3108815680126B6066B
:10BAD000B543156083F31088026E012A02D0FDF78A
:10BAE000ABF870BD0466EFF31083012282F3108877
:10BAF000026815681024A543156083F31088026856
:10BB0000D369DB43DB0600D41462098BFCF7CAFD62
:10BB100070BD000000480040F8B504460025904F75
:10BB200020682269A168E369114362691A431143DD
:10BB300002688C4B1A400A43026020684168032265
:10BB400012039143E26811434160A0692168B94240
:10BB500001D0226A10438A680B231B029A430243D6
:10BB60008A608149226881488A4213D1C06880076F
:10BB7000800F07D0012809D0022805D0032807D05C
:10BB8000102142E0012140E002213EE004213CE09E
:10BB900008213AE076498A4213D1C0680C21084056
:10BBA00007D0042809D0082805D00C2807D0102178
:10BBB0002BE0002129E0022127E0042125E00821D3
:10BBC00023E06C498A4201D100211EE06A498A4281
:10BBD00001D1002119E0BA4216D1C06803218902BF
:10BBE00008400BD001218902401A0BD0401A07D01F
:10BBF000884201D1082108E0102106E0002104E07C
:10BC0000022102E0042100E010215D485B4E830028
:10BC1000BA4236D1002913D0022914D0042917D0F2
:10BC2000082918D000200125002861D06268510041
:10BC30005118814202D8110381420FD2012589E0B7
:10BC4000FBF7FEFEF0E73168C906EDD41846EBE7D6
:10BC5000FBF716FFE8E70120C003E5E7010E060247
:10BC60005008002330185941F9F758FA0321090206
:10BC7000444A411A914202D82168C8606AE001250D
:10BC800068E00122E769D203974234D1092919D229
:10BC90000F007F443F79FF19BF4404070A140F14B3
:10BCA00014141200FBF7CCFE0EE0FBF7D9FE0BE0FC
:10BCB0003168C90608D4184606E0FBF7E1FE03E048
:10BCC000104601E000200125002843D061684000B3
:10BCD0004A088018F9F70CFA02462B49103A8A42B2
:10BCE00007D8491C01400007420F0A432068C26080
:10BCF00030E001252EE0092919D20F007F443F7959
:10BD0000FF19BF4404070A140F1414141200FBF7A0
:10BD100097FE0EE0FBF7A4FE0BE03168C90608D4DD
:10BD2000184606E0FBF7ACFE03E0104601E00020F9
:10BD3000012500280ED061684A081018F9F7D8F9D3
:10BD40000146114A1039914203D8216880B2C86077
:10BD500000E001250020A066E0662846F8BD00004E
:10BD600000480040F369FFEF0038014040100240F6
:10BD700000440040004C00400050004000100240D1
:10BD800000093D00FFFC0F00EFFF000070B5044606
:10BD900061655820025300212546803569602220C4
:10BDA0002860606F002819D0214BC362636F21485F
:10BDB0001863636F20485863606F81632168666D04
:10BDC000134624313246606FFAF7F3FF002805D09E
:10BDD0001020686020202860012070BD20690028A4
:10BDE0000CD0EFF31081012080F3108820680268E6
:10BDF000FF2301331A43026081F31088EFF31081AF
:10BE0000012080F310882068836801221343836037
:10BE100081F31088EFF3108182F310882068826824
:10BE200040231A43826081F31088002070BD000017
:10BE3000A5B700083FB8000859B7000870B44165BD
:10BE4000014640310A834A830024846601238268C4
:10BE50001B03FF259A4207D10269002A01D08D8376
:10BE600019E02B4A8A8316E07F26002A09D0012593
:10BE70002D07AA420ED10269002A09D03F228A83E7
:10BE800009E00269002A01D08E8304E08D8302E07C
:10BE90008E8300E08C83014680314C6022220A6050
:10BEA000EFF31082012181F3108801688C6801256D
:10BEB0002C438C6082F310888168994202D1016919
:10BEC000002912D0134981660169002910D0EFF3CF
:10BED0001081012282F3108800680268FF23213359
:10BEE0001A43026081F310880EE00B498166EBE78C
:10BEF000EFF31081012282F310880068026820238A
:10BF00001A43026081F3108870BC00207047000063
:10BF1000FF0100003DBA000861B9000810B4C16F0C
:10BF2000212910D1014640314A8A002A0DD0C26C25
:10BF300003681288D205D20D9A62C26C921CC26448
:10BF4000488A401E488210BC7047EFF310820121DE
:10BF500081F3108801680B688024A3430B6082F38F
:10BF60001088EFF31081012282F3108800680268C4
:10BF700040231A43026081F3108810BC704710B44C
:10BF8000C16F21290ED1014640314A8A002A0BD0C7
:10BF9000C26C036812789A62C26C521CC264488AEE
:10BFA000401E488210BC7047EFF31082012181F3DC
:10BFB000108801680B688024A3430B6082F310880B
:10BFC000EFF31081012282F3108800680268402399
:10BFD0001A43026081F3108810BC7047FFB583B02C
:10BFE0000C9D04460E4617462068C16930468843BA
:10BFF00027D00020B84245D120468030029020381A
:10C000000190681C36D0FBF70DF90699401AA8423A
:10C0100019D8002D17D02068016849072AD5C169B1
:10C02000C943090712D42068082505622046FFF796
:10C0300041FC02984560019900200876012007B074
:10C04000F0BD0120D6E7032007B0F0BDC069C043B2
:10C0500000050FD401202168C00208622046FFF7C6
:10C0600029FC0298202141600199002008760320D4
:10C0700007B0F0BD2068C1693046884305D0002074
:10C08000B842BED0002007B0F0BD0120F8E70000A4
:10C0900010B50248FCF72EFB10BD0000CC040020B8
:10C0A00010B50248FCF726FB10BD00005405002027
:10C0B000F8B51D4D0E0034D0032832D27421484308
:10C0C0001A494418A078002802D0012822D028E07C
:10C0D000E168A068421860680090406F006840689E
:10C0E0002769101A0818C01BF9F702F8012905D8AA
:10C0F00017D100980068C069800612D43878307073
:10C1000061692069884201D1A06800E0401C20617B
:10C11000002506E0204618303146FCF7F3FE0028E3
:10C12000F6D02846F8BD0000FFFFFFFF2C280020B6
:10C1300070B50C00064601D0032E02D30020C04388
:10C1400070BD7421484321490E54227845186A7005
:10C150006078A8706068A860A168E9606278002AC9
:10C1600002D0012A05D00BE028614018401E68610A
:10C1700006E0284618300123A2686168FCF79DFE9E
:10C18000E068E86220692863A069286760696863DD
:10C190002078002801D0012806D121460C310EC993
:10C1A00028463830FDF71BFB6078002804D00128B2
:10C1B00006D0022804D006E0304600F009F802E07C
:10C1C000304600F021F8002070BD00002C2800202F
:10C1D00038B50C497422504342185068016804E095
:10C1E0004C6A6B461C801C881C80CB691B07F7D4EB
:10C1F00091681161D368CC18641E54619AB2FCF73F
:10C20000B3FC38BD2C28002074214843044910B5E4
:10C2100040180146683140680122FCF7D9FC10BD86
:10C220002C28002070B5054674201A49684344182C
:10C23000A078002802D0012807D00DE0A068206176
:10C24000E1684018401E606106E020461830012376
:10C25000E268A168FCF731FE6078002801D001286F
:10C2600006D121462C310EC920463830FDF7B7FAE9
:10C27000A078002804D0012806D0022804D006E0C7
:10C280002846FFF7A5FF02E02846FFF7BDFF002084
:10C2900070BD00002C28002070B50D0001D00328CF
:10C2A00002D30020C04370BD7421484304494418A0
:10C2B00074212046FDF7B4F80020656070BD0000D1
:10C2C0002C28002010B502460E4900207423434359
:10C2D0005B185B6893420FD17422424351188978EE
:10C2E000002906D0012901D0022901D1FFF78CFFD6
:10C2F00010BDFFF76DFF10BD401CC0B20328E5D391
:10C3000010BD00002C28002038B501461348002439
:10C3100074226243121852688A4219D1742161430F
:10C320000818817801290BD0022908D1016F002952
:10C3300002D0806EC0B288472046FFF765FF38BD47
:10C34000816E6A46117069461830FCF79BFDF3E771
:10C35000641CE4B2032CDBD338BD00002C28002081
:10C36000F7B582B00021009103991546002903D04A
:10C37000002D01D0032803D30020C04305B0F0BD39
:10C38000742148432B4946187078344638340028C5
:10C3900004D0012820D0022842D049E0FCF796FEC4
:10C3A00020462946FDF7EDF9070033D020463946EF
:10C3B000FDF7B3F92A4638680399F8F7DFFE2046FF
:10C3C000FDF7C1F90446FDF70FF8A088216882B295
:10C3D0007068FCF7A7FC2BE0FCF778FE20462946A6
:10C3E000FDF7CFF9070015D020463946FDF795F93E
:10C3F0002A4638680399F8F7C1FE2046FDF7A3F9ED
:10C400000446FCF7F1FFA088216882B27068FCF74F
:10C41000E3FC0DE0FCF7E8FF0020C043009007E0DC
:10C42000134664204343AAB270680399FCF709FCE1
:10C430000098A3E72C28002070B51F4A0021742320
:10C440004B439B185B68834231D1742041438C1865
:10C450006078002816D0012813D1204638300546D0
:10C46000FDF771F901462846FDF741F92846FDF729
:10C470006AF9002805D081888AB201686068FCF7F3
:10C48000ABFC70BD204638300546FDF75CF901462F
:10C490002846FDF72CF92846FDF755F90028F0D07D
:10C4A00081888AB201686068FCF73CFC70BD491C59
:10C4B000C9B20329C3D370BD2C280020F8B53E4C67
:10C4C000002321783D4A1D46082910D0072947D06E
:10C4D000062950D0052952D0042953D0032954D01D
:10C4E000002956D0012958D002295AD05BE0A17802
:10C4F00000264A1F04E0314FBF5DFB189BB2761C3B
:10C500009642F8DB667927799A195118E3786278B0
:10C51000C9188918C9194018C0430006000E1AD15D
:10C52000012E14D0022E16D125482449C018F8F740
:10C5300025FE00F0F7FE642000F01FFDBFF34F8FD3
:10C5400021492048C860BFF34F8F00BFFDE759085D
:10C550001046FEF7AFFB2570E570A570A571F8BD1C
:10C56000A1795054491CC8B2A071A178491F8842D2
:10C57000F5D1082001E0607007202070F8BDE07060
:10C580000620FAE760710520F7E7A070E570042047
:10C59000F3E7552807D10120EFE7AA2803D10220AD
:10C5A000EBE7032803D02570E570A570F8BD0320E4
:10C5B00020702071F8BD000078000020740A00206F
:10C5C000740600200400FA0500ED00E07CB5154675
:10C5D000024600201C4600290BD0491E0092019102
:10C5E000044B6A462146284600F020F9009A0021B3
:10C5F00011707CBD65CF00082021020C01D01021F4
:10C600001046020A01D010460839020901D010462E
:10C61000091F820801D01046891E420801D0881ED9
:10C620007047081A7047F0B4040C8BB2264682B2E9
:10C630005E430D0C1046370C584336048019002118
:10C64000794116466E43370C3604801979412646E7
:10C650006E438919F0BC7047BFF34F8F04490348FC
:10C66000C860BFF34F8F00BFFDE700000400FA056C
:10C6700000ED00E0BFF34F8F04490348C860BFF3EB
:10C680004F8F00BFFDE700000400FA0500ED00E059
:10C6900000487047B403002002E008C8121F08C118
:10C6A000002AFAD170477047002001E001C1121F33
:10C6B000002AFBD170470000F0B51FB486B009987E
:10C6C000089A030D0021024314D05148514A18180A
:10C6D000504305141198012810981AD0281A401CAC
:10C6E00000264D4F4D49009601910490002812DA22
:10C6F000444211E01198012449A3012801D1109866
:10C70000C1430698119A84600360C26041600BB017
:10C71000F0BD4042E4E70446210500203F4A001CEA
:10C7200051410391029012E0E00707D032463B46A8
:10C7300001990098F8F70EFF0191009032463B46B0
:10C7400010461946F8F706FF06460F466410002CFF
:10C75000EAD10498039B0028029A0999089806DAFE
:10C76000F8F7F8FE019B009AF8F7F4FE05E0F8F7F9
:10C7700059FF019B009AF8F755FF04460E46002228
:10C78000284BF9F71BF803D80020C043014607E007
:10C790000022254B20463146F8F72AFEF9F74AF9E0
:10C7A000102409E0002C0ADB0A220023F8F7B6FC6B
:10C7B000079B30321A55641E02460A43F2D11122F9
:10C7C000641C079B121B1C19119B012B03D0012316
:10C7D00008430ED10AE0084304D011201090002035
:10C7E000119077E71098151A6D1E0BE01098824291
:10C7F00002DD00236D1C03E0824201DA00236D1E7E
:10C80000002BEED0069811998260C16030C07EE79F
:10C8100001FCFFFF104D0000000014400000F03F3D
:10C82000300000000000F0430000E03FFFB597B08B
:10C830000646002518E2252877D100242746FD4921
:10C84000049400E00443761C32780120203A9040A2
:10C850000842F7D130782A280ED0022230780146DB
:10C860003039092916D804990A2359433039401818
:10C870001443761C0490F1E7189802C804911890AC
:10C88000002904DA012040030443484204900220B6
:10C890000443761C30782E2814D104200443707889
:10C8A000761C2A2809D11898761C80C8189009E0AF
:10C8B0000A214F43303FC719761C30780146303982
:10C8C0000929F5D930786C2810D006DC4C281AD00C
:10C8D00068280ED06A2817D104E0742813D07A286B
:10C8E00012D110E00120400504430CE001210905AC
:10C8F00001E0032109050C437178814203D1012035
:10C9000000052418761C761C3078119066280BD010
:10C9100013DC58287DD009DC00287BD04528F6D0D0
:10C920004628F4D047281AD1A5E118E0632835D06D
:10C93000642870D0652812D19DE170286CD008DC85
:10C940006728F1D069287BD06E280DD06F2806D1DA
:10C95000BAE073282ED0752871D0782859D01A9A49
:10C96000199990476D1C7EE16002400F022809D0A2
:10C9700003280DD00428189801680DD00D60001D03
:10C98000189070E11898EA1701680D604A60F6E7A0
:10C99000189801680D80F2E70D70F0E718986A4664
:10C9A00001781172001D18900020507202A80090AA
:10C9B000012005E0189802C8189000200091C0439B
:10C9C00061070DD5002101E00199491C0191B9428F
:10C9D00012DA8142F8DB009A515C0029F4D10BE0B5
:10C9E000002101E00199491C01918142FADB019A81
:10C9F0000099895C0029F5D1019904981A9B471A7E
:10CA000021463846199A00F097FA019940194518BD
:10CA10000BE04FE02CE113E04EE000980099007825
:10CA2000491C00911A9A199990470198401E01904B
:10CA3000401CF2D1214638461A9B199A10E137E082
:10CA40000A200021009001916002410F022907D0C5
:10CA5000189A01CA1892C2179446032908D00AE00E
:10CA60001898C01DC108C90005C91891944607E06F
:10CA700000B2C2179446042902D140B2C1178C46B5
:10CA800000226146944506DA0A460021404291415F
:10CA90008C462D2102E0210504D52B216A46117315
:10CAA000012103E0E10701D02021F7E7029155E0E1
:10CAB0000A200AE0102008E0102000900021042045
:10CAC00004430191082703E0082000210191009010
:10CAD0006002410F022907D0189A01CA1892002259
:10CAE0009446032908D008E01898C01DC108C90061
:10CAF00005C91891944603E080B2042900D1C0B260
:10CB000000210291210729D51199702906D0009A98
:10CB10001021019B4A401A4305D00EE040216A468D
:10CB20001173012108E06146014306D030216A46B5
:10CB300011731199517302210291009A0821019BEE
:10CB40004A401A430AD16146014301D1610705D524
:10CB500030216A46117301217F1E029111995829D3
:10CB600004D035A10E910DA90D910DE037A1F9E783
:10CB70006146019B009AF8F7D1FA0E9B8C469B5CAC
:10CB80000D9A521E0D92137061460143F0D10D981B
:10CB900005A9081A20300190600703D50120000480
:10CBA000844300E001270198874201DD381A00E044
:10CBB0000020019900904118029809180498401A21
:10CBC0000490E00306D421461A9B199A049800F0B9
:10CBD000B3F94519002706E003A81A9AC05D199910
:10CBE00090476D1C7F1C02988742F5DBE0030CD553
:10CBF00021461A9B199A049800F09EF9451904E001
:10CC00001A9A3020199990476D1C0099481E00907F
:10CC10000029F5DC08E00D980D990078491C0D916C
:10CC20001A9A199990476D1C0199481E0190002984
:10CC3000F1DC63E109280100303132333435363715
:10CC40003839616263646566000000003031323358
:10CC500034353637383941424344454600000000F8
:10CC600000F05AF94519761C3078002800D0E2E52A
:10CC700028461BB0F0BD600700D406271898C01DD9
:10CC8000C108C90048680A680831C30FDB0718915A
:10CC9000190001D09CA108E0210501D59BA104E069
:10CCA000E10701D09AA100E09AA1430011985B0826
:10CCB000109165280CD006DC452809D046281DD0E7
:10CCC000472841D141E0662818D067283CD13CE094
:10CCD0000021112F01DB112000E0781C0191009050
:10CCE00008A911A8FFF7E8FC139905910021119AF2
:10CCF00015927F1C12980197009150E00120C00707
:10CD000003900120019008A9009711A8FFF7D4FC17
:10CD1000139A149905920022119B00921298159370
:10CD2000059A0192002901D0104602E0791C4018B2
:10CD30000190381A01D5019804E04042401E00904D
:10CD4000781C0190C01B029043E0012F00DA0127FC
:10CD50000021112F01DD112000E0384601910090E3
:10CD600008A911A8FFF7A8FC13990591119A0021B1
:10CD7000129815920091019721070CD40599B94298
:10CD800001DB019900E00191012904DD159A491E9A
:10CD9000515C302906D0B84201DA011D05DA0121C3
:10CDA000029115E00199491EEDE7002805DC009984
:10CDB000411800910199091A03E0019A411C91421E
:10CDC00000DD01910099401A401C02900120C0072B
:10CDD0000390200706D402990198814202DB0020CB
:10CDE000C043029000206946C87707AF012103982D
:10CDF0000337C907884224D0022011902B201290BB
:10CE0000039800280CDA404203902D20129007E08E
:10CE10000A210398F8F76CF930317F1E03903970BE
:10CE20001199481E11900029F2DC03980028EFD1D7
:10CE3000791E129808703078202108404530BF1EB6
:10CE4000387006A8C01BC01D0390109800780028F9
:10CE500000D00120019941180298C01709180398C1
:10CE600009180498401A401E0490E00306D4214695
:10CE70001A9B199A049800F05FF8451910980078E9
:10CE8000002803D01A9A199990476D1CE00324D505
:10CE900021461A9B199A049800F04EF845191CE097
:10CEA0000098002807DB00990598884203DD159853
:10CEB000405C199901E0199930201A9A904700981E
:10CEC0006D1C401C00900298401E0290002804D166
:10CED0001A9A2E20199990476D1C0199481E0190AD
:10CEE0000029DDDC05E038781A9A7F1C19999047F3
:10CEF0006D1C0399481E03900029F4DC21461A9BFF
:10CF0000199A0498ACE600002D0000002B000000E8
:10CF10002000000000000000F8B5044600251E4671
:10CF20001746880404D405E039462020B0476D1C1C
:10CF3000641EF9D52846F8BDFFB50446002581B02A
:10CF40001E46C80301D5302700E02027880404D5F9
:10CF500005E038460399B0476D1C641EF9D5284694
:10CF600005B0F0BD4A68002A06D00A68531C0B6061
:10CF700010704868401E486070477D2110B5C90098
:10CF8000484300F001F810BD002140E000BF00BFA1
:10CF900000BF00BF00BF00BF00BF00BF00BF00BF99
:10CFA00000BF00BF00BF00BF00BF00BF00BF00BF89
:10CFB00000BF00BF00BF00BF00BF00BF00BF00BF79
:10CFC00000BF00BF00BF00BF00BF00BF00BF00BF69
:10CFD00000BF00BF00BF00BF00BF00BF00BF00BF59
:10CFE00000BF00BF00BF00BF00BF00BF00BF00BF49
:10CFF00000BF00BF00BF00BF00BF00BF00BF00BF39
:10D0000000BF00BF00BF00BF00BF00BF491C81427E
:10D01000BCD37047FAF722F9FEF766F9FDF72EF94F
:10D02000FDF7F4F8FDF7CCF9FDF75CFAFDF776FAB9
:10D03000FDF7E2F9FDF706FA1E481D4901600021DF
:10D040004160816001621C4A416242618162FAF77B
:10D05000E3F9002801D072B6FEE7FDF757FBF8F7B9
:10D0600095FFF8F777FEFDF77DFEFDF775FAFF20D7
:10D07000000203461A461146FDF758FEFF24F53418
:10D080002046F9F7CFFEFF20000403461A4611465A
:10D09000FDF74CFE2046F9F7C5FE0124074DF8F7D1
:10D0A00081FEAC70F9F72CF8FEF76EFAF7E7000096
:10D0B000007C004014040020FFFF0000000000205E
:10D0C00010B50446FCF74EFC4E20FCF71DFCFCF7A7
:10D0D00085FCE0B2FCF718FCFCF780FCFCF742FC96
:10D0E0004F20FCF711FCFCF779FC0020FCF7DEFB7D
:10D0F0000446FCF753FC204610BD70B50D460446AF
:10D10000FCF730FC4E20FCF7FFFBFCF767FCE0B2BD
:10D11000FCF7FAFBFCF762FC2846FCF7F5FBFCF792
:10D120005DFCFCF73BFC0A20FFF72EFF70BD000002
:10D1300010B52421002000F04DF81B48FFF724FF14
:10D1400000210F2000F046F80521102000F042F8E1
:10D150000421112000F03EF883217F2000F03AF8EE
:10D1600069217F2000F036F8BD217F2000F032F8E1
:10D170000E480078262804D1002240218C2000F09F
:10D1800019F8012000F02AF8094814210187282005
:10D1900000F020F80A20FFF7F7FE012000F036F833
:10D1A000012000F043F810BD204E0000D800002000
:10D1B00074060020F8B517460E4605460024FFF712
:10D1C0007FFF3946B44331402143284600F002F83E
:10D1D0000020F8BD10B5FFF790FF10BD10B5002876
:10D1E0000AD000212720FFF7F5FF04211920FFF7BF
:10D1F000F1FF8721162005E000211620FFF7EAFF46
:10D2000000211920FFF7E6FF10BD000010B500282F
:10D2100001D0002200E0802280211120FFF7CAFF08
:10D220000148FFF7B1FE10BDA086010010B500282F
:10D2300011D001212F20FFF7CDFF62213020FFF711
:10D24000C9FF46213120FFF7C5FF32210846FFF70D
:10D25000C1FFA22100E022213320FFF7BBFF10BD58
:10D260000C480D4A0188914210D1C18832290DD352
:10D27000C18E43290AD8818F012907D8C08F012880
:10D2800004D8044840308088012801D90120704723
:10D290000020704774060020AA55000010B5012434
:10D2A000A40221461948F7F782FF22461749184879
:10D2B000F9F776F81548174902888A4224D0018088
:10D2C000154981801549C1800A23038100214181CC
:10D2D00081810122C28181834324C4860224048780
:10D2E0000F4C44878287C2870246403211845184A2
:10D2F0009184C1839180142484821182E1210901E7
:10D300008184038400F00EF810BD00007406002034
:10D3100000FC0008AA55000034120000102700008D
:10D320003C0F000070B5FFF79BFF002801D00120E3
:10D3300070BD72B60124074DA40221462846F9F7B4
:10D3400015F8002804D0224603492846F9F7B4F816
:10D3500062B670BD00FC000874060020002100E0E9
:10D36000491C8142FCD3704734D50008D3B2000871
:10D370001CD5000819B00008F4D4000805AF000857
:10D38000D8D4000841AE0008ACD40008E9AD0008CC
:10D390000CD50008B9AF000814D50008BDAF0008CF
:10D3A00098D4000825B0000804D50008C9B10008C9
:10D3B000A0D4000821B10008CCD4000849B200086C
:10D3C00024D50008C1B00008ECD40008CDAE000898
:10D3D000C4D4000895AE0008E4D40008B1AD00083C
:10D3E000B8D4000879AD0008FCD40008C9B2000820
:10D3F0000000000000000000010203040607080905
:10D40000030406080C10182030000000000102037D
:10D410000400404040404040404040414141414183
:10D4200040404040404040404040404040404040FC
:10D43000404005020202020202020202020202024D
:10D440000202202020202020202020200202020290
:10D4500002020290909090909010101010101010F6
:10D4600010101010101010101010101010020202E6
:10D47000020202888888888888080808080808083E
:10D48000080808080808080808080808080202022E
:10D490000240000012D400087365745F6164630089
:10D4A0007365745F6465765F6964000064656275C6
:10D4B000675F6F6666000000626565705F6F666635
:10D4C000000000006770735F6F6666007365745FCD
:10D4D000776966690000000064656275675F6F6E5A
:10D4E00000000000626565705F6F6E006770735FBB
:10D4F0006F6E0000696E666F00000000736C6565FA
:10D50000700000007365745F697000007274635F7F
:10D51000676574007274635F736574007265626F2F
:10D520006F7400007365745F636F6E7472617374FF
:10D530000000000074657374000000002B2B2B0D9D
:10D540000000000061742B6A6F696E3D6F74616149
:10D550002C31300D0000000061742B63683D636E58
:10D560003437302C330D000061742B64723D350D5F
:10D570000000000061742B6170706575693D353283
:10D5800036393733363936653637343834360D0068
:10D5900061742B636C6173733D610D0061742B6169
:10D5A00070706B65793D32623765313531363238AE
:10D5B00061656432613661626637313538383039D9
:10D5C0006366346633630D0061742B6D6F64653D73
:10D5D0006D61630D0000000061742B6164723D6F2A
:10D5E00066660D0061742B7265626F6F740D0000CA
:10D5F00061742B736C6565703D6C696768742C3061
:10D600002C6C6576656C2C6C6F770D0061742B64E7
:10D6100065766575693D3437333635343966303073
:10D620003331253034780D00636C65617200000081
:10D630006C73000054D6000800000020B8030000FE
:10D64000645B0008B0D60008B8030020E82C000096
:10D65000A8C60008014F4350011204125002238053
:10D66000392DF90B31BA0C0F133CD51B08C8041A1D
:10D6700044041A9004130CD61B0874081A9C041A4C
:10D6800068041A58041AD8041AF0041AE404410A67
:10D6900025277F9204021D2032021A287813FD905C
:10D6A0001B0830084BB1916801FF01FF0172720144
:04000005080050C1DE
:00000001FF
